:100000000C94DB070C9403080C9403080C9403086D
:100010000C9403080C9403080C9403080C94030834
:100020000C9403080C9403080C94901A0C94FF1A77
:100030000C9403080C9403080C9403080C94030814
:100040000C9403080C9403080C9403080C94030804
:100050000C9403080C9403080C9403080C94311DB1
:100060000C9403080C9403080C9403080C940308E4
:100070000C9403080C9403080C9403080C940308D4
:100080000C9403080C9403080C9403080C940308C4
:100090000C9403080C9403080C9403080C940308B4
:1000A0000C9403080C9403080C9403084461790031
:1000B00041636374004C6F616E00436170616369FA
:1000C0007479200047756E732000050512151F1501
:1000D0000905082466E766244120596573202042FB
:1000E000204E6F000042726F6F6B6C796E00436F31
:1000F0006E65792049736C616E64004D616E686154
:100100007474656E0043656E7472616C2050617228
:100110006B0047686574746F0042726F6E78000000
:100120004C7564657300537065656400576565645C
:100130000041636964004865726F696E6500436FD2
:100140006361696E65002000200003081F051F1F02
:10015000151B1F11111F110E1F15111F05011F1156
:100160001D1F041F001F0010101F1F041B1F101055
:100170001F061F1F011F1F111F1F05071F311F1FF4
:10018000051B17151D011F011F101F0F100F1F0C3E
:100190001F1B041B071C071915130C121E1F120C22
:1001A0001E12120C121F0C1A14041F052E2A1E1FD9
:1001B000021C001D00201D001F041A011F001E0448
:1001C0001E1E021E1E121E3E120C0C123E1E0206A7
:1001D00014120A020F121E101E0E100E1E081E1AF6
:1001E000041A2E281E1A12161F111F001F001D159B
:1001F0001711151F07041F17151D1F151D01011FBE
:100200001F151F17151F00170000100020100000F9
:10021000030004083E09093E3F25251A1E2121122C
:100220003F21211E3F2525213F0505011E21293A99
:100230003F04043F213F21001021211F3F040A31C8
:100240003F2020203F02023F3F02043F1E21211E8B
:100250003F0909061E21112E3F09093622252519BD
:10026000013F01011F20201F0F10201F3F10103FD2
:100270003B04043B03043807312D2321102A2A3C78
:100280003F2424181C2222141824243F1C2A2A2C20
:10029000047E05014C52523E3F040438243D2000A8
:1002A0004040443D3F081422213F20003E04043ECC
:1002B0003E04023C1C22221C7E22221C1C22227E86
:1002C0003E040204242A2A12021F22201E20201E7D
:1002D0000E10201E3E10103E360808364E50503E7E
:1002E000322A26221E29251E223F200032292926B5
:1002F0001221251A0C0A3F08172525191E25251835
:10030000013905031A25251A0629291E002F000088
:10031000002000004020000000030000000000005A
:10032000003E5B4F5B3E3E6B4F6B3E1C3E7C3E1C7B
:10033000183C7E3C181C577D571C1C5E7F5E1C00C1
:10034000183C1800FFE7C3E7FF0018241800FFE778
:10035000DBE7FF30483A060E2629792926407F053B
:100360000507407F05253F5A3CE73C5A7F3E1C1C51
:1003700008081C1C3E7F14227F22145F5F005F5F11
:1003800006097F017F006689956A606060606094FD
:10039000A2FFA29408047E040810207E2010080802
:1003A0002A1C08081C2A08081E101010100C1E0C0D
:1003B0001E0C30383E3830060E3E0E06000000009F
:1003C0000000005F00000007000700147F147F1486
:1003D000242A7F2A122313086462364956205000CB
:1003E00008070300001C2241000041221C002A1CB7
:1003F0007F1C2A08083E08080080703000080808A2
:100400000808000060600020100804023E514945C1
:100410003E00427F400072494949462141494D33DF
:100420001814127F1027454545393C4A4949314146
:10043000211109073649494936464949291E000014
:100440001400000040340000000814224114141469
:100450001414004122140802015909063E415D5955
:100460004E7C1211127C7F494949363E414141225E
:100470007F4141413E7F494949417F090909013E88
:10048000414151737F0808087F00417F41002040AF
:10049000413F017F081422417F404040407F021CC1
:1004A000027F7F0408107F3E4141413E7F090909D8
:1004B000063E4151215E7F091929462649494932A4
:1004C00003017F01033F4040403F1F2040201F3F6A
:1004D0004038403F631408146303047804036159EF
:1004E000494D43007F414141020408102000414131
:1004F000417F0402010204404040404000030708DD
:100500000020545478407F284444383844444428D8
:10051000384444287F385454541800087E0902187F
:10052000A4A49C787F0804047800447D4000204007
:10053000403D007F1028440000417F40007C04784B
:1005400004787C080404783844444438FC18242493
:100550001818242418FC7C08040408485454542413
:1005600004043F44243C4040207C1C2040201C3C90
:100570004030403C44281028444C9090907C446487
:10058000544C44000836410000007700000041361A
:10059000080002010204023C2623263C1EA1A161A0
:1005A000123A4040207A38545455592155557941D2
:1005B0002154547841215554784020545579400CA9
:1005C0001E5272123955555559395454545939558A
:1005D0005454580000457C410002457D42000145CD
:1005E0007C40F0292429F0F0282528F07C5455453A
:1005F000002054547C547C0A097F493249494932CD
:100600003248484832324A4848303A4141217A3AE1
:1006100042402078009DA0A07D39444444393D40AB
:1006200040403D3C24FF2424487E4943662B2FFC58
:100630002F2BFF0929F620C0887E09032054547906
:10064000410000447D413048484A32384040227AD7
:10065000007A0A0A727D0D19317D2629292F282654
:100660002929292630484D4020380808080808085C
:100670000808382F10C8ACBA2F102834FA00007BB5
:10068000000008142A142222142A140895002200BB
:1006900095AA005500AAAA55AA55AA000000FF0075
:1006A000101010FF00141414FF001010FF00FF10B2
:1006B00010F010F0141414FC001414F700FF0000E4
:1006C000FF00FF1414F404FC141417101F10101F63
:1006D000101F1414141F00101010F0000000001F51
:1006E000101010101F10101010F010000000FF105C
:1006F0001010101010101010FF10000000FF140058
:1007000000FF00FF00001F10170000FC04F4141489
:100710001710171414F404F40000FF00F714141455
:1007200014141414F700F7141414171410101F10D5
:100730001F141414F4141010F010F000001F101FF8
:100740000000001F14000000FC140000F010F01066
:1007500010FF10FF141414FF141010101F000000DD
:1007600000F010FFFFFFFFFFF0F0F0F0F0FFFFFFE1
:100770000000000000FFFF0F0F0F0F0F3844443838
:10078000447C2A2A3E147E02020606027E027E0273
:1007900063554941633844443C04407E201E200692
:1007A000027E020299A5E7A5991C2A492A1C4C72CF
:1007B00001724C304A4D4D303048784830BC625A56
:1007C000463D3E494949007E0101017E2A2A2A2AE6
:1007D0002A44445F444440514A444040444A5140C2
:1007E0000000FF0103E080FF000008086B6B083683
:1007F00012362436060F090F0600001818000000F4
:100800001010003040FF0101001F01011E00191DE2
:100810001712003C3C3C3C0000000000D5F08D1459
:10082000A1C881CFD9F1AF20005810F0F89C8E8775
:1008300083878E9CF8F00000FEFF03030303030789
:100840000EFCF80000FEFF0303030303070EFCF891
:100850000000FFFF00000000000000FFFF0000FE9E
:10086000FF8383838383C7EE7C380000F8FC0E0788
:10087000030303070EFCF800003F7FE0C08080C048
:10088000E07F3FFFFF01010101010101FFFF0000C7
:10089000FFFF0C0C0C0C1C3E77E3C100007FFFC077
:1008A000C0C0C0C0E0703F1F00001F3F70E0C0C06C
:1008B000C0E0703F1F00007FFFC1C1C1C1C1E3772D
:1008C0003E1C00001F3F70E0C0C0C0E0703F1F0032
:1008D0000000000001FFFF01000000486172646138
:1008E0007373272063617263617373212100646FE6
:1008F0006C6C617273206F6E204F666669636572FF
:10090000007468656D2120596F7520666F756E647F
:100910002000596F75206B696C6C656420616C6C8C
:10092000206F6600596F75206B696C6C6564206F71
:100930006E65212100002020596F75206D69737349
:10094000656421212100006861766520746F207242
:10095000756E2100616E792067756E732120596F65
:100960007500596F7520646F6E2774206861766515
:10097000007468656D2100596F752063616E27747E
:10098000207368616B6500616E20616C6C65792114
:100990002100596F75206C6F7374207468656D2029
:1009A000696E00756E697473206F663A2000596F26
:1009B0007520666F756E642000323030206275637A
:1009C0006B733F006D6F726520706F636B6574733E
:1009D00020666F72007472656E6368636F61742065
:1009E000776974680057696C6C20796F752062753F
:1009F000792061206E65770057696C6C20796F757E
:100A000020736D6F6B652069743F006C696B6520A6
:100A1000676F6F6420737475666621210068657264
:100A200065207468617420736D656C6C7300546824
:100A3000657265277320736F6D6520776565640047
:100A4000646F6C6C6172733F007370656369616C95
:100A500020666F7220343030007361747572646187
:100A600079206E69676874002E3434206D61676E7A
:100A7000756D20666F7200626172657474612066C4
:100A80006F720034303020646F6C6C6172733F00A1
:100A900057696C6C20796F752062757920610061EF
:100AA0006674657220796F7521006465707574696C
:100AB00065732061726500206F662068697300614C
:100AC0006E6420004F6666696365722048617264D7
:100AD00061737300696E2074686520737562776155
:100AE000792100596F752077657265206D7567678C
:100AF000656400617265206F7574726167656F75FA
:100B0000732121212100636F6B652062757374214D
:100B1000205072696365730050696773206D61646A
:100B200065206120626967007072696365732121C5
:100B300021006174206F7574726167656F75730051
:100B4000627579696E67206865726F696E650041CC
:100B50006464696374732061726500726169642101
:100B60002121210066726F6D206C6173742077659E
:100B7000656B2773006368656170206865726F69D3
:100B80006E650050696773206172652073656C6CD7
:100B9000696E6700626F74746F6D6564206F757441
:100BA0002121210057656564207072696365732097
:100BB00068617665006C7564657321212100736539
:100BC0006C6C696E6720636865617000526976615C
:100BD0006C206465616C6572732061726500746F6E
:100BE0006461792100626F72726F776564206D6F46
:100BF0006E657900596F7520616C7265616479006A
:100C00002100596F7520646F6E27742068617665C6
:100C100020616E7900004F6F707321002100596FC1
:100C2000752063616E2774206166666F72640000D0
:100C30004F6F7073210021006D6F72652000596F36
:100C4000752063616E277420636172727900004FB2
:100C50006F70732100457874656E64656420476128
:100C60006D653A00004E6F726D616C2047616D6575
:100C70003A00596F7527726520646561642121000F
:100C80006265656E206869742100596F7527766505
:100C9000006D69737365642121005468657900797A
:100CA0006F75212120005468657927726520666977
:100CB00072696E672061740041204669676874201C
:100CC00020422052756E004552524F522000004F74
:100CD0006C642000486967682053636F72653A004E
:100CE0000047616D65206F766572212053636F72D6
:100CF000653A00416D7400536176696E67730059FF
:100D00006F75206F776500596F7520686176650093
:100D10005769746864726177204D6F6E657900441D
:100D200065706F736974204D6F6E657900426F72E4
:100D3000726F77204D6F6E657900506179204C6F2E
:100D4000616E000000517479005072696365004360
:100D50006F73747300596F75206861766500536511
:100D60006C6C20004275792000000075703F0064B3
:100D70006F63746F7220746F2073657720796F755D
:100D800000646F6C6C61727320666F722061005733
:100D9000696C6C20796F752070617920313030304A
:100DA00000596F7572206865616C74683A20007331
:100DB00074696C6C20616674657220796F752100AE
:100DC00020706967730054686572652061726520E0
:100DD000004265696E672063686173656421210064
:100DE0005769746864726177204D6F6E657900444D
:100DF00065706F736974204D6F6E65790042616E26
:100E00006B00426F72726F77204D6F6E6579005282
:100E100065706179204C6F616E004C6F616E20537C
:100E20006861726B004A65742066726F6D200053B2
:100E3000656C6C204472756773004275792044724A
:100E4000756773005472656E6368636F6174004206
:100E5000616E6B004C6F616E20536861726B004A6B
:100E60006574005472656E6368636F6174005365E6
:100E70006C6C2044727567730042757920447275FA
:100E8000677300486967682053636F726573004534
:100E90007874656E6465642047616D6500486974A7
:100EA0002074686520537472656574730076312E02
:100EB000322E3000536C616E67696E27001E1E0073
:100EC00000C0800000000000000000807807067865
:100ED00080000000000000000000C040000000038F
:100EE0003CC10204081020C000FF00000000FF0009
:100EF000C02010080404C2390700003850909090B8
:100F00002324485060812608E70090E70826016006
:100F1000504826A19090905030000000000001023F
:100F200022322A2422100A080C081221242A320212
:100F300003000000000000080B000202020000098C
:100F40000400000102020000052400100105240134
:100F5000010104240206052406000107058103108F
:100F6000004009040100020A0000000705020240D7
:100F70000000070583024000000403090412010079
:100F800002EF0201404123368000010102030141CA
:100F9000726475696E6F204C4C43004172647569D0
:100FA0006E6F204C656F6E6172646F0003051F0EDB
:100FB0000400AE1D7C3011241FBECFEFDAE0DEBF8F
:100FC000CDBF12E0A0E0B1E0E0E3FEE602C0059094
:100FD0000D92AE34B107D9F727E0AEE4B2E001C01C
:100FE0001D92A039B207E1F717E0CAEDD7E004C0BF
:100FF0002197FE010E940A35C93DD107C9F70E9419
:101000002F1E0C940B370C940000E2EEF2E0A0E0EF
:10101000B8E000800EBC8111012C1197A0FDFDCF1E
:101020000192B9F70DB40895480F592F511D1416A8
:10103000150684F5803891056CF597FF02C090E0A5
:1010400080E04138510514F040E850E0481BFB01B6
:10105000E770FF2721E001C0220FEA95EAF777FF4A
:1010600002C0695F7F4FFB0133E0F595E7953A9544
:10107000E1F7F695FE2FEE27F795E795E80FF91FB4
:10108000EE51FD4F415030F08191DF011197822BDD
:101090008C93F8CF08956F927F928F929F92AF9228
:1010A000BF92CF92DF92EF92FF920F931F93CF9355
:1010B000DF93DC017A014115510509F49CC0FA0166
:1010C000149131965491F2E0EF0EF11CC12FD0E053
:1010D000222309F1CC24C394D12C852F877011F4DD
:1010E000D12CC12CE52FE695E695E695EC0DFD2D6E
:1010F000F11DEC9FC001ED9F900DFC9F900D112400
:10110000033011F4880F991F289FF001299FF00DDB
:101110001124EE0EFF1EFD01EC0FFD1F1E161F0613
:101120000CF069C0A038B1050CF065C0CB01850F8B
:10113000911D181619060CF05EC0603471050CF094
:101140005AC0E114F10409F456C0362F3770CB01B0
:1011500077FD079623E0959587952A95E1F7282F47
:1011600077FF04C0332311F02FEF280F662777276E
:101170006A1B7B0BB7FD02C070E060E090E89A1B31
:10118000E038F1050CF4912F961BE22F022E000C93
:10119000FF0BDE2ED0942F3F0CF0D12C41E0852F99
:1011A000877009F440E0B52EB694B694B6944B0D12
:1011B000E40FF11D399714F048E0421BB42EBD181E
:1011C0002D0D40E82403F0011124AE0FBF1FA60F20
:1011D000B71F1D9D600D711D1124A701460F571FDC
:1011E000C32E032E000CDD08033009F4C7C090F4B1
:1011F000023009F474C0DF91CF911F910F91FF90DD
:10120000EF90DF90CF90BF90AF909F908F907F90A6
:101210006F9008950A3FA1F1B20E0B3F61F72B15B5
:1012200051F3BD016E517D4F10E000E0091708F049
:101230009FC0FA01E00FF11FE491F0E04F010C2C88
:1012400002C0880C991C0A94E2F727FD06C0FB0136
:101250008081F82CF0948F218083332361F0273034
:1012600054F47B01F0E8EF0EF11CA92CA094F701D7
:1012700080818A2180830F5F1F4F6F5F7F4FD6CFA2
:10128000B20E2B1509F4B7CFBD016E517D4F10E0A2
:1012900000E0091708F066C0FA01E00FF11FE491C1
:1012A000F0E04F010C2C02C0880C991C0A94E2F764
:1012B00027FD04C0FB01808188298083332351F0FE
:1012C000273044F47B01F0E8EF0EF11CF701808138
:1012D000892980830F5F1F4F6F5F7F4FDACF6FEFDA
:1012E00070E0032E02C0660F771F0A94E2F7609544
:1012F0007095972E8B2C820E281509F47CCF8D01CA
:101300000E511D4FF12CE12CE91630F5FA01EE0DCE
:10131000FF1DE491F0E03F010C2C02C0660C771C2D
:101320000A94E2F727FD05C0F8018081862386290B
:101330008083332359F027304CF45801F0E8AF0E86
:10134000B11CF5018081892187298083FFEFEF1A85
:10135000FF0A0F5F1F4FD8CF2F5F4C0F5D1FA058A4
:10136000BF4FCACF2F5F4C0F5D1FA058BF4F89CF13
:101370002F5F4C0F5D1FA058BF4F51CFE92EF12CAE
:10138000FA01E60FF71FAE51BD4F60E870E06E192D
:101390007F09CE19DF098E01000F111F41E050E0D7
:1013A0007A01032E01C0EE0C0A94EAF7592F4B2D57
:1013B000892E932ECF93DF93ED01EF96EF96229631
:1013C000A590C590992059F0AE9C5001CE9C60012B
:1013D00027302CF4F880D094FD20FB28F9922223AA
:1013E0003AF0FC90C094FC20FA28FD920C94F90984
:1013F00011965A9529F74A9551F0582D23951124A5
:10140000E00FF11DA60FB11DC60FD11DD9CFDF9181
:10141000CF911124F0CE0F9302E020E00E944B0800
:101420000F9108952F923F924F925F926F927F9209
:101430008F929F92AF92BF92CF92DF92EF92FF92E4
:101440000F931F93CF93DF93CDB7DEB728970FB6D7
:10145000F894DEBF0FBECDBF6F836A0119011C83F4
:101460000B83FE82ED82811128C005E010E029E0A7
:1014700030E03A832983B6010D2C000C880B990BC0
:101480000E94BB314B015C015F8151111DC0E0E541
:10149000F7E090E080E018861F828C159D050CF027
:1014A0002BC1248135814F8158854217530714F48D
:1014B00038872F8301963696F0CF04E010E048E09D
:1014C00050E05A834983D7CF20E030E040E05FE32B
:1014D0000E941A324B015C0120E030E0A9010E9419
:1014E000F53420E030E040E05FE387FD30C0C50127
:1014F000B4010E9489330E94673478876F83A60104
:101500008F819885481B590BE0E5F7E090E080E07B
:10151000B12CA12C2F81388582179307ECF086E03F
:10152000829FF001839FF00D1124E05BF84F90E063
:1015300080E0D12CC12C84179507BCF4248135811F
:10154000C216D3060CF4690101963696F4CFC50194
:10155000B4010E948833CFCF24813581A216B3060F
:101560000CF4590101963696D5CFB801110F880BAE
:10157000990B0E94BB312B013C01B5016C0D7D1D07
:10158000072E000C880B990B0E94BB3120E030E045
:1015900040EE5FE30E9489336B017C0120E030E084
:1015A00040E05FE3C301B2010E941A329B01AC012B
:1015B000C701B6010E941A326B017C0120E030E0C5
:1015C000A9010E94F53420E030E040E05FE387FDB0
:1015D00089C0C701B6010E9489330E94673402E4C2
:1015E00010E0061B170BF10111830083B501BB0C42
:1015F000880B990B0E94BB3120E030E040EE5FE3A6
:101600000E948933A30192010E941A324B015C01AE
:1016100020E030E0A9010E94F53420E030E040E015
:101620005FE387FD64C0C501B4010E9489330E9455
:101630006734600F711FEB81FC81718360832981A6
:101640003A81B901330F880B990B0E94BB3120E01E
:1016500030E040E05FE30E941A326B017C014F8171
:101660005885BA01550F880B990B0E94BB319B011D
:10167000AC01C701B6010E941A326B017C0120E067
:1016800030E0A9010E94F53420E030E040E05FE363
:1016900087FD85C0C701B6010E9489330E94673467
:1016A0002AE230E0C901861B970BED81FE81918310
:1016B000808328960FB6F894DEBF0FBECDBFDF91B2
:1016C000CF911F910F91FF90EF90DF90CF90BF903F
:1016D000AF909F908F907F906F905F904F903F90D2
:1016E0002F900895C701B6010E94883376CFC501B7
:1016F000B4010E9488339BCFB801110F880B990B5E
:101700000E94BB3120E030E040E05FE30E941A32EB
:101710002B013C01EF81F885BF01FF0F880B990B6E
:101720000E94BB319B01AC01C301B2010E941A327D
:101730002B013C0120E030E0A9010E94F53420E0BB
:1017400030E040E05FE387FD25C0C301B2010E94A5
:1017500089330E94673422E430E0C901861B970B6D
:10176000F101918380838FEF9FEFEB81FC81918367
:10177000808329813A81B901330F880B990B0E942C
:10178000BB3120E030E040E05FE30E941A32A50167
:10179000940171CFC301B2010E948833DACFC7012F
:1017A000B6010E9488337ACFFC018091E102882340
:1017B00011F13FB7F89482E08093E9002091F200A4
:1017C000822F90E01816190614F481E090E0882327
:1017D00039F0289844E64093E0024091F1004083BC
:1017E000222339F02091F200211103C02BE620932F
:1017F000E8003FBF08958FEF9FEF08952FB7F8944B
:1018000083E08093E9009091E800892F807295FF32
:1018100004C09091F20080E4891B2FBF089580914D
:10182000D80281110DC082E08093D40284E08093BD
:10183000D5021092D7021092D60281E08093D8028E
:1018400084ED92E00895CF93DF931F92CDB7DEB77A
:101850006983DC01ED91FC910280F381E02D41E090
:1018600050E0BE016F5F7F4F09950F90DF91CF91E0
:10187000089583E08093E9008091F200882319F0B5
:101880008AE38093E80008950E94FE0B90E008959B
:10189000CF93DF931F92CDB7DEB7FC01848595858A
:1018A00097FD08C02FEF3FEF358724870F90DF911A
:1018B000CF910895CE0101960E94D40B019719F49F
:1018C000898190E0F3CF8FEF9FEFF0CF0F931F93BD
:1018D000CF93DF931F92CDB7DEB78C01FC018485D7
:1018E000958597FF0BC0CE0101960E94D40B0197FE
:1018F00071F4898190E0F80195878487F8018485E7
:1019000095850F90DF91CF911F910F9108958FEFE3
:101910009FEFF1CFFC018485958597FD0BC09FB7A4
:10192000F89482E08093E9008091F2009FBF90E0FC
:10193000019608959FB7F89482E08093E900809122
:10194000F2009FBF90E008954091CE025091CF02E7
:101950002091CC023091CD0242175307B4F49091FC
:10196000E8009570E1F39091E80092FD19C0809332
:10197000F1008091CE029091CF0201968F7399274A
:10198000892B19F48EEF8093E8008091CE0290911C
:10199000CF0201969093CF028093CE0281E008950A
:1019A00080E00895DF92EF92FF920F931F93CF9301
:1019B000DF93D82E8A01EB017B01E40EF51ECE15D4
:1019C000DF0559F0D7FE12C0FE0184910E94A40CDD
:1019D00021968111F4CF0FEF1FEFC801DF91CF9156
:1019E0001F910F91FF90EF90DF9008958881EECFC7
:1019F0000F931F93CF93DF931F92CDB7DEB782E093
:101A0000898342E450E067E37FE080E80E94D20CE3
:101A10000E940F0CDC0112960D911C91011511050D
:101A200089F0D801ED91FC910280F381E02DBE0197
:101A30006F5F7F4FC801099597FD04C0F8010085CD
:101A40001185ECCF89810F90DF91CF911F910F917C
:101A50000895615030F02091F100FC01208301963F
:101A6000F8CF289884E68093E00208953FB7F89471
:101A70008091C8029091C902A091CA02B091CB0294
:101A800026B5A89B05C02F3F19F00196A11DB11DD9
:101A90003FBFBA2FA92F982F8827BC01CD01620F15
:101AA000711D811D911D42E0660F771F881F991FD0
:101AB0004A95D1F708958F929F92AF92BF92CF929D
:101AC000DF92EF92FF926B017C010E94360D4B0179
:101AD0005C01C114D104E104F104B9F00E94360D97
:101AE000681979098A099B09683E73408105910547
:101AF00080F321E0C21AD108E108F10888EE880ECF
:101B000083E0981EA11CB11CE4CFFF90EF90DF9002
:101B1000CF90BF90AF909F908F9008958F929F929B
:101B2000AF92BF92CF92DF92EF92FF920F931F93EB
:101B3000CF93DF936C017B018A018091140188238C
:101B400009F45CC08091E102882309F457C08091B8
:101B5000D30280FF05C08091E00082608093E000A6
:101B6000E801B12C8AEFA82E93E0892E2AE3922E69
:101B7000209711F4BB20D9F10E94FE0B81110AC0FD
:101B8000AA94AA20D9F161E070E080E090E00E9480
:101B90005B0DEECF8C171D0611F00CF08C2F9FB74C
:101BA000F8948092E9002091E80025FD02C09FBFD3
:101BB000DFCF282F30E0C21BD30BF701815020F07C
:101BC00041914093F100FACFE20EF31EBB2021F0C9
:101BD0009092E800B12CEBCF8091E80085FDE7CF33
:101BE0009092E800BB24B394209709F3F3CF5D985B
:101BF00084E68093D202101611063CF081E090E05A
:101C0000F6019383828310E000E0C801DF91CF9159
:101C10001F910F91FF90EF90DF90CF90BF90AF900A
:101C20009F908F9008950895DB0114964D915C91DB
:101C300015976D917C91DC01ED91FC910280F3810F
:101C4000E02D09942F923F924F925F926F927F9274
:101C50008F929F92AF92BF92CF92DF92EF92FF92BC
:101C60000F931F93CF93DF9300D000D000D0CDB758
:101C7000DEB7782E662E5A0128E0422E512C8111B3
:101C800003C099E0492E512CCE0101967C018E01B2
:101C90000D5F1F4F9E012B5F3F4FA501662D872DC6
:101CA0000E94120AB5010B2C000C880B990B0E94A4
:101CB000BB3120E030E040E05FE30E941A326B016C
:101CC0007C0120E030E0A9010E94F53420E030E002
:101CD00040E05FE387FD24C0C701B6010E9489335D
:101CE0000E9467348B0180E5C82E87E0D82E049DC2
:101CF0001001059D300C149D300C1124F12CE12CA9
:101D0000912C812C8A149B04B4F589819A816620D8
:101D100019F0801691064CF42D818E0D9F1D0BC07D
:101D2000C701B6010E948833DBCF2B81A70142197E
:101D30005309840F951F7720A1F0209379072093F2
:101D4000780780937A07B60184E797E00E94140E23
:101D50009FEF891A990A86E0C80ED11CE40CF51C85
:101D6000D1CF209383072093820780938407B60105
:101D70008EE797E0EBCF26960FB6F894DEBF0FBE46
:101D8000CDBFDF91CF911F910F91FF90EF90DF902A
:101D9000CF90BF90AF909F908F907F906F905F900B
:101DA0004F903F902F900895EF92FF920F931F93C3
:101DB000CF93DF938C017B01D0E0C0E0F701EC0F03
:101DC000FD1F6491662361F0D801ED91FC910190B3
:101DD000F081E02DC8010995892B11F02196EECFF5
:101DE000CE01DF91CF911F910F91FF90EF90089559
:101DF000AF92BF92CF92DF92EF92FF920F931F9319
:101E0000CF93DF936C017B018B01040F151FEB0156
:101E10005E01AE18BF08C017D10759F06991D6010D
:101E2000ED91FC910190F081E02DC6010995892B7F
:101E300079F7C501DF91CF911F910F91FF90EF903E
:101E4000DF90CF90BF90AF900895BC0190E080E00C
:101E50000C945B0D8FB18095807F669B88601C9B86
:101E60008460089590915602982329F49091570226
:101E7000982381E009F480E0089580389105B8F452
:101E800060347105A0F420E191E061FD94E060FD13
:101E9000990F62FD9295687F269FD0011124A80FAB
:101EA000AE51BD4F8C9140FF03C0892B8C93089598
:101EB00090958923FBCF2F923F924F925F926F9222
:101EC0007F928F929F92AF92BF92CF92DF92EF92CA
:101ED000FF920F931F93CF93DF937C016B018824B4
:101EE0008394912CD0E0C0E005E010E096EF692EDD
:101EF00077247A942CEFA22EBB24BA94842F84707A
:101F0000582E842F8270482E842F8870382E41706E
:101F1000242E219682E0880E911CA80CB91C552015
:101F200091F041E0B8016C0D7D1DC7018C0F9D1F24
:101F30000E943D0F41E0B6016C0F7D1FC8018E0D60
:101F40009F1D0E943D0F442091F041E0B601601BAF
:101F5000710BC7018C0F9D1F0E943D0F41E0B60120
:101F60006C1B7D0BC8018E0D9F1D0E943D0F332001
:101F700091F041E0B6016C0F7D1FC701801B910BF2
:101F80000E943D0F41E0B8016C0D7D1DC7018C1B07
:101F90009D0B0E943D0F222091F041E0B6016C1B89
:101FA0007D0BC701801B910B0E943D0F41E0B601E4
:101FB000601B710BC7018C1B9D0B0E943D0FC0174E
:101FC000D10754F4B7FCA5CF0150110982E0680E87
:101FD000711CA60CB71C9DCFDF91CF911F910F9163
:101FE000FF90EF90DF90CF90BF90AF909F908F9039
:101FF0007F906F905F904F903F902F9008952F9219
:102000003F924F925F926F927F928F929F92AF9288
:10201000BF92CF92DF92EF92FF920F931F93CF93D5
:10202000DF93EC0141E06FE370E00E943D0F41E07F
:1020300065E370E0CE010E943D0F41E06AE370E08D
:10204000CE0105960E943D0F41E06AE370E0CE01AB
:1020500005970E943D0F22242394312CF12CE12C72
:1020600005E010E036EF432E55245A944CEFC42E71
:10207000DD24DA948FEFE81AF80A82E0280E311C8A
:10208000C20CD31C47018C0E9D1E41E058018AE30F
:10209000A80EB11CB501C4010E943D0F3E016E188F
:1020A0007F0841E0B501C3010E943D0F41E08AE392
:1020B000A82EB12CA01AB10AB501C4010E943D0F8F
:1020C00041E0B501C3010E943D0F47018AE3880E3C
:1020D000911C41E0B4015E01A00EB11EC5010E9439
:1020E0003D0F41E0B4013E01601A710AC3010E9434
:1020F0003D0F9AE3892E912C8E189F0841E0B40180
:10210000C5010E943D0F41E0B401C3010E943D0F93
:10211000E016F1069CF0DF91CF911F910F91FF9097
:10212000EF90DF90CF90BF90AF909F908F907F9077
:102130006F905F904F903F902F900895D7FC9ACF6B
:102140000150110982E0480E511CC40CD51C92CFDD
:102150008F929F92AF92BF92CF92DF92EF92FF92B7
:102160000F931F93CF93DF936D3089F0C09054028B
:10217000D09055026A30D1F410925302109252025C
:1021800088E0C80ED11CD0925502C092540281E062
:1021900090E0DF91CF911F910F91FF90EF90DF9032
:1021A000CF90BF90AF909F908F9008950091520272
:1021B00010915302E5E06E9FE0011124C45EDC4FF4
:1021C0004801F12CF5E0E12CFF1629F0CE01019633
:1021D000FE01E490EC01B12CA12C4E2D4170B60112
:1021E0006A0D7B1DC4010E943D0FE694FFEFAF1AFC
:1021F000BF0A88E0A816B10481F7F394EFEF8E1AB6
:102200009E0AF6E0FF12DECF0A5F1F4F10935302C3
:1022100000935202BCCFDF92EF92FF920F931F9375
:10222000CF93DF937C01D22E8B01040F111DEB01A4
:1022300077FF02C0D0E0C0E0C8010134110514F0FE
:1022400080E490E0C817D9073CF44D2DBE01C701CA
:102250000E943D0F2196F0CFDF91CF911F910F91FA
:10226000FF90EF90DF9008952F923F924F925F92F0
:102270006F927F928F929F92AF92BF92CF92DF9296
:10228000EF92FF920F931F93CF93DF9300D000D074
:1022900000D0CDB7DEB76C01762E542E4901602EEA
:1022A00098E0A92EB12C611103C089E0A82EB12CB1
:1022B000CE0101967C018E010D5F1F4F9E012B5FA9
:1022C0003F4FA401652D872D0E94120A09811A81B2
:1022D000552011F1B401990C880B990B0E94BB3168
:1022E00020E030E040E05FE30E941A321B012C0145
:1022F00020E030E0A9010E94F53420E030E040E029
:102300005FE387FD0CC0C201B1010E9489330E94C6
:102310006734C616D70644F48D809E8009C0C2017A
:10232000B1010E948833F3CF8B809C80C61AD70AF4
:10233000CA9CB001CB9C700DDA9C700D1124060F65
:10234000171FC40104976620B1F061E070E07110BE
:1023500002C062E070E0060F171F6C01C6012FEF8C
:10236000C21AD20AC814D90491F020E045E0B8019D
:102370000E940B11F3CF61E070E0711002C062E0C7
:1023800070E0600F711F4CEA5FE00E940B0A269616
:102390000FB6F894DEBF0FBECDBFDF91CF911F9176
:1023A0000F91FF90EF90DF90CF90BF90AF909F90F4
:1023B0008F907F906F905F904F903F902F900895F7
:1023C0000F93CF93DF93EC019E816A3059F48D8196
:1023D0008C836985960F9E8381E090E0DF91CF9199
:1023E0000F910895262F61E0690F2A3398F4203366
:1023F00078F5273249F140F4213261F198859C5FEC
:102400008C81890F8C83E8CF2C3231F12E32B1F7D9
:102410002FE309C0213490F32B35C0F08FE9820FF0
:1024200027548A3158F7062E000C770B8C81082E22
:10243000000C990B3F810AEF313009F00BEF42E1BC
:1024400052E00E944B08DACF21E4EDCF2154EBCFCC
:102450002C5FE9CF2EE3E7CF20E4E5CF0F93CF93B6
:10246000DF93EC019E816A3059F48D818C836985FC
:10247000960F9E8381E090E0DF91CF910F910895B8
:10248000262F61E0690F2A3398F4203378F527323C
:1024900049F140F4213261F198859D5F8C81890F6B
:1024A0008C83E8CF2C3231F12E32B1F72FE309C003
:1024B000213490F32B35C0F08FE9820F27548A31F5
:1024C00058F7062E000C770B8C81082E000C990B08
:1024D0003F810AEF313009F00BEF4AE451E00E94EE
:1024E0004B08DACF21E4EDCF2154EBCF2C5FE9CFBD
:1024F0002EE3E7CF20E4E5CFE8E9F2E080EB92E0DD
:1025000030E020E04191519161917191240F351F8C
:102510008E179F07B9F78091670290916802821B1E
:10252000930B0895E091BC02F091BD023197E73121
:10253000F10508F036C0E156FD4E0C940A35B6128E
:10254000D112BC12D112B912BF12C212D112D112C1
:10255000B612C512D112D112D112D112D112D1128A
:10256000CC12CC12D112B912D112B91282E090E081
:10257000089581E090E0089583E090E0089584E07C
:1025800090E0089585E090E008958091B2029091E6
:10259000B3020497029728F4809177029091780211
:1025A000089590E080E00895CF93C82F84E00E94C2
:1025B000320F811107C0CC23B1F088E00E94320FA6
:1025C000882389F01092C2020E9492129093C10255
:1025D0008093C0028091B2029091B3029093BD02A9
:1025E0008093BC0281E0CF910895E4E7F7E08AE4AC
:1025F0008583848387E3868368ED70E0CF010E9442
:10260000D40E8BE490E00E94FF0F87E690E00C94DC
:10261000FF0FCF92DF92EF92FF920F931F93CF9312
:10262000DF9346E770E060E085E090E00E941408E8
:1026300046E76FE370E085E090E00E94140821E037
:1026400046E365E070E090E080E00E940B1121E03D
:1026500046E365E070E08FE790E00E940B1141E0F7
:1026600065E070E085E090E00E945B0F42E065E08D
:1026700070E08AE790E00E945B0F44E06AE370E05C
:102680008AE790E00E945B0F48E06AE370E085E033
:1026900090E00E945B0F80917902C2E3D7E0811144
:1026A00022C00AE010E0F12CE12C8AE0C82ED12CE7
:1026B00080917A0290917B02E816F90684F58FEFFB
:1026C000E81AF80AD0925302C092520210935502AF
:1026D00000935402BE0188E897E00E94140E065F42
:1026E0001F4F2696E5CF1AE0F12CE12C0AE08091ED
:1026F0007A0290917B02E816F9068CF40093830726
:102700000093820710938407BE018EE797E00E9432
:10271000140E8FEFE81AF80A175F2696E8CFDF91BC
:10272000CF911F910F91FF90EF90DF90CF90089580
:10273000BC01EEE7F7E096E0958394838CE0868316
:10274000CF010C94140E90E080E008958F929F9238
:10275000AF92BF92EF92FF920F931F93CF93DF93AD
:10276000CDB7DEB7A1970FB6F894DEBF0FBECDBFD1
:102770007C01FA01CB0119A2223008F42AE08E0173
:102780000F5D1F4F822E912CB12CA12CBF01A501F2
:1027900094010E945733F901CA016A3074F5605DF3
:1027A000D8016E938D01232B242B252B79F790E0F4
:1027B00080E0109789F0FD0101900020E9F7319742
:1027C000AF014A1B5B0BD701ED91FC910280F381B5
:1027D000E02DB801C7010995A1960FB6F894DEBFA8
:1027E0000FBECDBFDF91CF911F910F91FF90EF9062
:1027F000BF90AF909F908F900895695CD1CFCF929A
:10280000DF92EF92FF920F931F93CF93DF9377FFA7
:1028100021C06A017B01EC01E881F9810190F0811E
:10282000E02D6DE209958C0144275527BA014C191A
:102830005D096E097F092AE0CE010E94A613800F70
:10284000911FDF91CF911F910F91FF90EF90DF903B
:10285000CF9008952AE0DF91CF911F910F91FF90C3
:10286000EF90DF90CF900C94A613CF93DF93CFE13E
:10287000D0E020E04AE067E170E0CE010E940B1159
:102880002196CF36D105A9F783E280938307809301
:10289000820788E18093840740916302509164022B
:1028A00060916502709166028EE797E0DF91CF91AB
:1028B0000C94FF13BC01EEE7F7E09AE09583948354
:1028C00088E18683CF010E94140E48E566E170E03E
:1028D0008EE190E00E94140848E561E270E08EE12C
:1028E00090E00E94140821E04CE066E170E08EE187
:1028F00090E00E940B1121E04CE066E170E085E77A
:1029000090E00E940B110E94351441ED50E068E107
:1029100070E08FE690E00C940B0ACF92DF92EF927A
:10292000FF920F931F93CF93C82F8B0169017A01F8
:102930006E5F7F4F4AEC50E00E940B0ACA5FEEE7E1
:10294000F7E0C583C4830683B701A601CF01CF9109
:102950001F910F91FF90EF90DF90CF900C94FF1399
:10296000CF93DF938091BC029091BD024297029772
:1029700068F5C8E2D0E020E047E065E270E0CE0113
:102980000E940B112196CF37D105A9F7E09177026C
:10299000F0917802EE0FFF1FEE0FFF1FE058FD4F82
:1029A0002081318142815381609163027091640280
:1029B00080916502909166020E94FA349B01AC01FD
:1029C00065E270E088E290E00E948D14DF91CF9183
:1029D0000C943514CF93DF93EC0188819981009793
:1029E00011F00E94AC35198218821D821C821B8254
:1029F0001A82DF91CF910895FC0180819181009727
:102A000011F00C94AC350895CF93C82F8091BA0281
:102A10009091BB0201969093BB028093BA021092F0
:102A200062020E94EB3021EE3EE240E050E00E9464
:102A3000EE326058714C8F4F9F4F609380027093BD
:102A4000810280938202909383020E94EB3029E5F9
:102A50003BE140E050E00E94EE3268577C4E8F4FE1
:102A60009F4F6093840270938502809386029093B7
:102A700087020E94EB3023E230E040E050E00E9409
:102A8000EE329B01AC01265F3F4F4F4F5F4FA4E6F4
:102A9000B0E00E940D3360938802709389028093A6
:102AA0008A0290938B020E94EB302BE230E040E0F0
:102AB00050E00E94EE329B01AC012F5D3F4F4F4F23
:102AC0005F4FAAE0B0E00E940D3360938C027093D8
:102AD0008D0280938E0290938F020E94EB3020E152
:102AE00030E040E050E00E94EE329B01AC01295FF3
:102AF0003F4F4F4F5F4FAAE0B0E00E940D3360930D
:102B000090027093910280939202909393020E949C
:102B1000EB3025E030E040E050E00E94EE329B01D7
:102B2000AC012F5F3F4F4F4F5F4FAAE0B0E00E94D4
:102B30000D33609394027093950280939602909364
:102B40009702CC23C1F160916F0270917002809165
:102B50007102909172020E94BB312DEC3CEC4CE86A
:102B60005FE30E941A320E949D340E946734609392
:102B70006F02709370028093710290937202609161
:102B80006B0270916C0280916D0290916E020E94B6
:102B9000BB3124E13EEA47E85FE30E941A320E941B
:102BA0009D340E94673460936B0270936C02809333
:102BB0006D0290936E021092C202CF91089522E0AE
:102BC00030E03093BD022093BC0240ED57E060E05E
:102BD00070E0409373025093740260937502709397
:102BE000760248E853E160E070E040936F02509352
:102BF0007002609371027093720210926B021092D5
:102C00006C0210926D0210926E021092B10210923C
:102C1000B00210926A021092690224E630E030930A
:102C200068022093670222E330E030937D02209314
:102C30007C02E8E9F2E0119211921192119222E0E5
:102C4000E03BF207C1F701969093B9028093B80276
:102C50001092BB021092BA0280E00C9404159F926D
:102C6000AF92BF92CF92DF92EF92FF920F931F939A
:102C7000CF93DF935C017B018B01D0E0C0E0F801D2
:102C800091908F016501CC0EDD1EC6010E94D832E5
:102C9000981621F0692DC6010E94E0322196C430B9
:102CA000D10569F7C701DF91CF911F910F91FF9077
:102CB000EF90DF90CF90BF90AF909F9008950C94CD
:102CC000D832CF92DF92EF92FF920F931F93CF9360
:102CD000DF93EB017B0124E0E20EF11C8B016C0120
:102CE000C61AD70AC601800F911F0E94D832F80178
:102CF00081938F01EE15FF05A9F7CE01DF91CF91EA
:102D00001F910F91FF90EF90DF90CF9008950F9358
:102D10001F93CF93DF938C01EB01FC0180819181A4
:102D20000097E1F06881798161157105A9F0428110
:102D300053812C813D814217530770F00E94043764
:102D40008C819D81F801958384831D821C82DF9193
:102D5000CF911F910F9108950E94AC358881998180
:102D6000F801918380838A819B81938382838C8104
:102D70009D8195838483198218821B821A82E5CFF4
:102D80000F931F93CF93DF93EC0188819981009774
:102D900059F02A813B812617370730F081E0DF9117
:102DA000CF911F910F9108958B016F5F7F4F0E940C
:102DB0003536009759F0998388831B830A832C81C9
:102DC0003D81232B59F7FC011082E8CF80E0E7CF4B
:102DD000EF92FF920F931F93CF93DF93EC017B0150
:102DE000CB010E944A310097A9F00C811D81080F88
:102DF000191FB801CE010E94C016882361F02881F6
:102E000039818C819D81B701820F931F0E944331CC
:102E10001D830C8381E0DF91CF911F910F91FF9073
:102E2000EF900895EF92FF920F931F93CF93DF934C
:102E3000FB01E080F180E114F10441F480E0DF91D6
:102E4000CF911F910F91FF90EF900895048115810C
:102E500001151105B1F0EC018C819D81080F191F3E
:102E6000B801CE010E94C016882341F32881398120
:102E70008C819D81B701820F931F0E9404371D83AF
:102E80000C8381E0DCCFEF92FF920F931F93CF93DF
:102E9000DF93EC018B016115710551F0CB010E94AC
:102EA0004A317C01BC01CE010E94C01681110BC0C9
:102EB000CE010E94EA14CE01DF91CF911F910F91B4
:102EC000FF90EF900895FD82EC82B801888199818E
:102ED0000E944331F0CFFC011182108213821282D2
:102EE000158214820C944317CF93DF93EC01623068
:102EF000710501F148F46115710581F061307105CA
:102F0000B1F06FE171E00CC064307105C9F0A8F058
:102F100065307105B1F760E271E002C06EE371E007
:102F2000CE010E946B17CE01DF91CF91089566E329
:102F300071E0F6CF61E371E0F3CF6CE271E0F0CFC6
:102F400066E271E0EDCFCF93DF93EC016230710563
:102F500001F148F46115710581F061307105B1F03E
:102F600064EE70E00CC064307105C9F0A8F0653003
:102F70007105B1F765EE70E002C069E171E0CE0164
:102F80000E946B17CE01DF91CF91089562E171E04D
:102F9000F6CF65E071E0F3CF6BEF70E0F0CF6EEE4F
:102FA00070E0EDCFEF92FF920F931F93CF93DF93DB
:102FB000EC017B018A01BA010E94C01681110BC08D
:102FC000CE010E94EA14CE01DF91CF911F910F91A3
:102FD000FF90EF9008951D830C83B701888199813C
:102FE0000E940437F0CFFB0101900020E9F73197F0
:102FF000AF01461B570B0C94D2170F931F93CF931F
:10300000DF93CDB7DEB762970FB6F894DEBF0FBE81
:10301000CDBF8C01CB01F801118210821382128284
:10302000158214824AE0BE016F5F7F4F0E945331C8
:10303000BE016F5F7F4FC8010E94F31762960FB603
:10304000F894DEBF0FBECDBFDF91CF911F910F91DE
:1030500008950F931F93CF93DF93CDB7DEB7A29759
:103060000FB6F894DEBF0FBECDBF8C01CB01BA0105
:10307000F8011182108213821282158214822AE0D2
:10308000AE014F5F5F4F0E945E31BE016F5F7F4FA9
:10309000C8010E94F317A2960FB6F894DEBF0FBEC8
:1030A000CDBFDF91CF911F910F9108952F923F9245
:1030B0004F925F926F927F928F929F92AF92BF9248
:1030C000CF92DF92EF92FF920F931F93CF93DF93F4
:1030D000CDB7DEB762970FB6F894DEBF0FBECDBF97
:1030E0002C019E012F5F3F4F490139011C01D12C5A
:1030F000C12C10E000E0B12CA12CF10141915191C3
:10310000619171911F01CE010D960E942918E988E5
:10311000FA88CE010D960E94FC14B601CE010D96E0
:103120000E94741789899A89E80EF91EFFEFEF1A39
:10313000FF0AF301E192F1923F01CE010D960E9448
:10314000FC14F3E0CF16D1040CF03FC0AE14BF0462
:103150000CF457012FEFC21AD20A36E0C316D1047D
:1031600061F680E5C82E87E0D82EF12CE12C150100
:1031700083E0E816F1040CF01801B701CE010D96BA
:103180000E947417BE01635F7F4FC6010E948716BD
:10319000CE010D960E94FC1468E471E0C6010E9405
:1031A000E816712C612CF401808191819101281B1A
:1031B000390B6216730674F466E471E0C6010E946E
:1031C000E8163FEF631A730AEECF0E151F0514F6CB
:1031D0008701C0CFF20141915191619171912F010D
:1031E000CE010D960E942918BE01635F7F4FC60174
:1031F0000E941217CE010D960E94FC14FFEFEF1AE9
:10320000FF0A26E0C20ED11C32E0830E911C86E03C
:10321000E816F10409F0ABCFF092B702E092B602E3
:1032200081E08093B4020A0D1B1D073111050CF4D7
:1032300080E08093B50262960FB6F894DEBF0FBEB1
:10324000CDBFDF91CF911F910F91FF90EF90DF9055
:10325000CF90BF90AF909F908F907F906F905F9036
:103260004F903F902F900895EF92FF920F931F93EE
:10327000CF93DF9300D000D000D0CDB7DEB78C0164
:103280009CE3E92EF12C20E04CE069E070E0C701FE
:103290000E940B118FEFE81AF80A80E8E816F10493
:1032A00091F7000F111F000F111FF801E856FD4F95
:1032B0004081518162817381CE0101960E9429185B
:1032C0008D818195880F880F845A80937907809328
:1032D00078078DE080937A0748E050E06CE571E074
:1032E00084E797E00E94F80EBE016F5F7F4F84E78E
:1032F00097E00E94140ECE0101960E94FC142696BF
:103300000FB6F894DEBF0FBECDBFDF91CF911F91F6
:103310000F91FF90EF900895EF92FF920F931F93FC
:10332000CF93DF9300D000D000D0CDB7DEB780912F
:10333000BC029091BD020A9709F05EC00E947C1207
:103340008C01BC01CE0101960E94FD17ED80FE802C
:10335000CE0101960E94FC1481E08093790780934E
:10336000780710927A0764EC70E084E797E00E9497
:10337000D40E4091690250916A02052E000C660B32
:10338000770B84E797E00E94FF1387E190E08E19A6
:103390009F09880F991F880F991F80937907809341
:1033A000780710927A076AEB70E084E797E00E9452
:1033B000D40EA801110F660B770B84E797E00E94EB
:1033C000FF1310E000E021E041E068E070E0C80198
:1033D0000E940B110F5F1F4F00381105A1F72696B1
:1033E0000FB6F894DEBF0FBECDBFDF91CF911F9116
:1033F0000F91FF90EF9008954091730250917402E5
:103400006091750270917602CE0101960E94291892
:10341000ED80FE80CE0101960E94FC1400E210E0D7
:103420000E191F09000F111F000F111F8091BC0200
:103430009091BD029C01265031092230310508F0DF
:1034400052C021E0209379072093780710927A07E1
:1034500060EB70E0069711F465EB70E084E797E0AD
:103460000E94D40E4AEC50E061E070E083E190E00D
:103470000E940B0A89E18093790780937807109264
:103480007A078091BC029091BD02069719F5409190
:103490006F0250917002609171027091720284E724
:1034A00097E00E94FF134AEC50E061E070E0C80131
:1034B00006970E940B0A00937907009378071092F1
:1034C0007A07409173025091740260917502709175
:1034D000760273CF40916B0250916C0260916D0245
:1034E00070916E02DCCF81E080937907809378073A
:1034F00010927A076CEA70E084E797E00E94D40E9D
:103500008EE0809379078093780710927A07409134
:10351000BA025091BB02052E000C660B770BBFCF91
:103520001F920F920FB60F9211248F939F93809149
:10353000E1009091E100937F9093E10083FF0FC041
:103540001092E90091E09093EB001092EC0092E36E
:103550009093ED001092E10298E09093F00082FFCA
:1035600022C093E09093E9009091F200992319F022
:103570009AE39093E8009091D202992341F09091C0
:10358000D20291509093D202911101C05D9A909114
:10359000E002992341F09091E00291509093E00273
:1035A000911101C0289A84FF18C08091E2008E7E9C
:1035B00081608093E2008091E1008F7E8093E10042
:1035C0008091D3028E7E80618093D3029F918F91F0
:1035D0000F900FBE0F901F90189580FFF7CF80912E
:1035E000E2008E7E80618093E2008091E1008E7E19
:1035F0008093E1008091D3028E7E8160E5CF1F929F
:103600000F920FB60F921124CF92DF92EF92FF929A
:103610000F931F932F933F934F935F936F937F93DA
:103620008F939F93AF93BF93EF93FF93CF93DF93CA
:10363000CDB7DEB76C97DEBFCDBF1092E9008091A9
:10364000E80083FF25C068E0CE0145960E94290D61
:1036500082EF8093E8008D8987FF39C09091E80060
:1036600090FFFCCF982F907609F034C19E894F8946
:10367000588D2F89F88C911131C0803861F5809177
:10368000D1028093F1001092F1008EEF8093E80058
:103690006C960FB6F894DEBF0FBECDBFDF91CF9111
:1036A000FF91EF91BF91AF919F918F917F916F911A
:1036B0005F914F913F912F911F910F91FF90EF904C
:1036C000DF90CF900F900FBE0F901F9018959EEF38
:1036D0009093E800C7CF1092F100D5CF913059F404
:1036E0008111D3CF4130510581F68091D1028D7F78
:1036F0008093D102CACF933049F48111C6CF4130B3
:10370000510519F68091D1028260F2CF953041F4D3
:103710008091E80080FFFCCF20682093E300B5CFC4
:10372000963009F0A9C00B8D1C8D22E01092E900A3
:103730001092CF021092CE02F2122EC01092CD0241
:103740001092CC020E94F80C1F8299E09983FA82B1
:1037500091E09E8390EA98879AEF99872091CE0214
:103760003091CF02275F3F4F3C832B838D83109294
:10377000E9001092CF021092CE021093CD02009376
:10378000CC0249E050E0BE016F5F7F4F80E00E94B5
:10379000D20C0E94F80C79CF1093CD020093CC028A
:1037A0000E940F0CDC0112960D911C910115110560
:1037B00009F451C1D801ED91FC910480F581E02D0F
:1037C000BE016B5E7F4FC8010995009709F03EC1AD
:1037D000F80100851185EACFF3E0FF120EC08F8952
:1037E000882309F440C0823061F440E860E18BE94D
:1037F0009FE00E947B1D811148CF81E28093EB0006
:1038000047CF813029F440E86BE08FE89FE0F1CFAB
:10381000833099F70E940F0CDC011296ED90FC901A
:103820008E010F5F1F4F6801E114F10479F0D70199
:10383000ED91FC910680F781E02DB801C701099553
:10384000080F111DF701E084F184EECFD8011C921E
:10385000F60101900020E9F73197BF016C197D094D
:1038600040E0C601C6CF69E77FE0FB01449150E02C
:1038700080E80E94D20C09CF973009F4BECF98306F
:1038800021F481E08093F10000CF993009F0FDCE62
:10389000837009F0B2CFE0E2F1E081E031E096E33D
:1038A0002191222371F08093E9003093EB00DF0136
:1038B00011972C912093EC009093ED008F5F87304F
:1038C00079F78EE78093EA001092EA008F8980935F
:1038D000E102DBCE8B8D9C8D1092E9001092CF021D
:1038E0001092CE029093CD028093CC02898D8111EB
:1038F00092C08E899D89913A49F4813209F07DCF39
:1039000047E050E06DE071E080E0B3CF913209F024
:1039100074CF833269F48F89988DB0E0A0E08093F2
:10392000090190930A01A0930B01B0930C01ADCE55
:10393000803269F48091E80082FFFCCF67E08DE07F
:1039400091E00E94290D8BEF8093E8009ECE823299
:1039500009F09BCE8F8980931401EEEFFFE78591EC
:1039600094918B3F9C4D51F1E0E0F8E080910D0186
:1039700090910E01A0910F01B0911001803B9440F5
:10398000A105B105F1F48091140180FD1AC0EE3F4C
:103990008AE0F80789F587E797E79183808380912C
:1039A00060008093D00288E19BE00FB6F894A89560
:1039B000809360000FBE9093600067CEEEEFFAE058
:1039C000D5CF808191818737974709F05ECEA89542
:1039D000809160008861809360008091D002809324
:1039E0006000EE3F2AE0F20789F08091FE0A909194
:1039F000FF0A9183808349CE808191818737980720
:103A000051F29093FF0A8093FE0AC5CF1092FF0AED
:103A10001092FE0A3ACE0E940F0CDC0112960D9114
:103A20001C910115110509F4E8CED801ED91FC9126
:103A30000190F081E02DBE016B5E7F4FC8010995BA
:103A4000811123CEF80100851185EBCF18161906D8
:103A50000CF41BCED2CEF1E0FF12BECE6DE77FE0BC
:103A600004CF1F920F920FB60F9211242F933F9302
:103A70008F939F93AF93BF938091C4029091C5029F
:103A8000A091C602B091C7023091C30223E0230F78
:103A90002D3758F50196A11DB11D2093C3028093C7
:103AA000C4029093C502A093C602B093C70280914E
:103AB000C8029091C902A091CA02B091CB020196AE
:103AC000A11DB11D8093C8029093C902A093CA02A0
:103AD000B093CB02BF91AF919F918F913F912F9166
:103AE0000F900FBE0F901F90189526E8230F029697
:103AF000A11DB11DD2CFEF92FF920F931F93CF93D1
:103B0000DF93F82E192FE62E042F81E0860F880F01
:103B10000E94A40C83E00E94A40CCF2DD12FEC0EA8
:103B2000FD2EF11CCE15DF05B9F007FF13C0FE0115
:103B300084910E94A40C182F80E00E94A40C812381
:103B400021968111EFCFDF91CF911F910F91FF90BF
:103B5000EF9008958881EDCF81E0F5CFCF93DF938B
:103B60001092E5061092E40688EE93E0A0E0B0E043
:103B70008093E6069093E706A093E806B093E906E3
:103B80008AE291E09093E3068093E2068FEF9FEF45
:103B90009093EF068093EE0610928B0710928A079F
:103BA00084E591E0909389078093880710928107BC
:103BB0001092800788E491E090937F0780937E07BE
:103BC00098E09093870781E080938607109283079F
:103BD00010928407109282078093850710927707CE
:103BE000109276072CE331E0309375072093740729
:103BF00090937D0780937C071092790710927A0743
:103C00001092780780937B07C0E5D7E0198218826D
:103C10001B821A821D821C8250E040E064E671E043
:103C2000CE010E94D217269687E0C437D80771F7D5
:103C3000C2E3D7E0198218821B821A821D821C827D
:103C400050E040E064E671E0CE010E94D217269673
:103C500087E0C035D80771F7DF91CF910895CF93F2
:103C6000DF93CDB7DEB72D970FB6F894DEBF0FBE4A
:103C7000CDBF789484B5826084BD84B5816084BDF5
:103C800085B5826085BD85B5816085BD80916E00FA
:103C9000816080936E00109281008091810082602B
:103CA0008093810080918100816080938100809168
:103CB0008000816080938000809191008260809379
:103CC000910080919100816080939100809190009B
:103CD0008160809390008091C10084608093C100D6
:103CE0008091C10082608093C1008091C100816099
:103CF0008093C1008091C30081608093C300809154
:103D0000C00082608093C0008091C2008160809377
:103D1000C20080917A00846080937A0080917A005A
:103D2000826080937A0080917A00816080937A002B
:103D300080917A00806880937A001092E10210925C
:103D4000D1021092D3028091D70081608093D70076
:103D500080EA8093D80089B5806189BD89B5826089
:103D600089BD09B400FEFDCF61E070E080E090E025
:103D70000E945B0D8091D8008F7C80618093D80079
:103D80008091E000807F8093E0008091E1008E7E52
:103D90008093E1008DE08093E200559A209A81ECB7
:103DA00080937C0085B1806F85B984B1877E84B9AA
:103DB00084B1876E84B95E9A5F988AB1806D8AB942
:103DC000769A6E9881B3806F81BB899880B38D702D
:103DD00080BB80E58CBD81E08DBD85E090E00E94D8
:103DE000250F5F9A85E090E00E94250F5E985C9811
:103DF000ECE1F8E089E298E024912EBD00000DB4DA
:103E000007FEFDCF31968E179F07B1F75C9A81E8C8
:103E1000809364008091650081608093650081E0FB
:103E200090E00E945F1681FF0EC0082F0470F02EF4
:103E300082FD2E9801EF1FEF0E942A0F86FF83C09C
:103E40002E9A2F9A2D9A82E480930001809164002B
:103E50008E7F8093640080917A00806480937A00E2
:103E600080917A0086FDFCCF009178001091790056
:103E70000E94360DAB01BC01C801B0E0A0E0DC013E
:103E8000992788276C017D01C40ED51EE61EF71EFA
:103E9000C701B60120916400216020936400611580
:103EA00071058105910511F00E943A311092BD0211
:103EB0001092BC021092C2028E010F5F1F4F780158
:103EC00001E110E07E2C6F2CC8010E94D832D7018E
:103ED0008D937D010F5F1F4F06311105A9F765E630
:103EE00071E0872D962D0E94FB3615E6E12E11E03C
:103EF000F12E01E110E0892B09F07EC065E071E050
:103F000086E190E00E94611661E071E08AE190E054
:103F10000E9461168FB7F8944091C4025091C50277
:103F20006091C6027091C7028FBF809150028823B2
:103F300009F480C01092500280E090E0892B51F388
:103F40000E940000E7CFFF2029F00430110511F492
:103F50002E9A2F9881E00E94050849E258E0B801A6
:103F600084E190E00E940B0A80E00E9405088FE047
:103F700090E00E94250F0F5F1F4F0931110509F0D6
:103F80005BCFFF2011F02F9A2D9880E991E00E94DD
:103F9000250F2D9A81E090E00E945F1680FF53CF9D
:103FA0008AE090E00E945F169FEF980F9E3F08F016
:103FB0004ACF22E330E0309353022093520228E3A9
:103FC00030E030935502209354020BE010E0682F4C
:103FD00088E897E00E94A810C8010E945F160F5F52
:103FE0001F4F0131110599F780E00E94050888EE06
:103FF00093E00E94250F27CFF701D1907F01C801E0
:104000000E94D832D81621F06D2DC8010E94E032EE
:104010000F5F1F4F0631110579F765E071E086E10A
:1040200090E00E942F1661E071E08AE190E00E942A
:104030002F1670CF80915102F42FF81B8F2F909183
:104040000001F91748F48F5F891708F075CF81E0F8
:1040500083BF889513BE70CF81E080935002409358
:10406000510280914E0290914F02019690934F021F
:1040700080934E0280915702809356020E942A0F2D
:10408000809357028091C2028111E4C02091BC024A
:104090003091BD02E2EEF2E081118FEF00248193B6
:1040A0008193819381930394D1F7109255021092DA
:1040B000540210925302109252028091C0029091C9
:1040C000C1029093BF028093BE021092C10210926F
:1040D000C0022230310589F42091BA023091BB022E
:1040E0008091B8029091B9022817390734F088E11D
:1040F00090E09093BD028093BC028091BC029091AD
:10410000BD028931910508F083C5FC01E657FF4DDA
:104110000C940A35A32005215121FB21C121C12185
:1041200075229F22B8221B23A221A823A823A823FB
:10413000A823B423E0237D23FF23FF23A124A1246C
:10414000A124A1240E254DEB5EE070E060E090E03C
:1041500080E00E940B0A4DEB5EE070E060E082E6DA
:1041600090E00E940B0A8AE290E0909353028093C1
:1041700052028AE090E0909355028093540264EBDF
:104180007EE088E897E00E94D40E87E68093790766
:10419000809378078AE380937A076DEA7EE084E76C
:1041A00097E00E94D40E6DE97EE080E597E00E94E2
:1041B00043176FE87EE086E597E00E94431763E8C7
:1041C0007EE08CE597E00E94431783E090E09093B7
:1041D000B7028093B60281E08093B5021092B402D8
:1041E00043E050E060E00E94220E2091B602309140
:1041F000B70200E04091B4026091B5028091BE0226
:104200009091BF020E94341122C00E940913209194
:10421000050130910601409107015091080163E1C9
:1042200070E08AE090E00E948D14209101013091AD
:104230000201409103015091040167E270E08AE0BD
:1042400090E00E948D141092B3021092B20281E0AD
:104250008093C202C090BC02D090BD02B9E1CB16DF
:10426000D10408F077C5F601E85CFE4D0C940A35E0
:104270002526572C252625262526252625262526AE
:10428000E32C572C572C572C5B2C5B2C5B2C572C7E
:10429000572C5B2CDC2DDC2DDC2DDC2DDC2DDC2DDE
:1042A000572C0E948C196091B0027091B102872D39
:1042B000962D0E94A317872D962D0E949813872D67
:1042C000962D0E94FC1469E77EE080E597E00E944D
:1042D00043176EE67EE086E597E00E94431763E6AB
:1042E0007EE08CE597E00E9443176FE57EE082E672
:1042F00097E00E9443178091B0029091B102892B00
:10430000F1F464E57EE088E697E00E9443176FE4ED
:104310007EE08EE697E00E94431786E090E090935F
:10432000B7028093B6021092B50281E08093B40286
:104330004091B6025091B70261E080E054CF84E032
:1043400090E0EDCF0E948C1964E47EE0872D962DDD
:104350000E946B17872D962D0E949813872D962DFE
:104360000E94FC1488E992E00E9456184091B6021F
:104370005091B7026091B4028091B5020E94220E62
:1043800066CF0E948C198091BC029091BD026AE3B5
:104390007EE0049711F06FE27EE0872D962D0E945B
:1043A0006B17872D962D0E949813872D962D0E94AE
:1043B000FC1480E892E00E9456184091B602509199
:1043C000B7026091B4028091B5020E94220EE09083
:1043D000BE02F090BF022091B6023091B70200E019
:1043E0004091B4026091B502C7010E943411C70127
:1043F0000E9434192CCF0E948C1965E27EE0CE0118
:1044000007960E946B176091B0027091B102872DE0
:10441000962D0E94A317672D762DCE0107960E9438
:104420001217872D962D0E94FC141A8219821C8265
:104430001B821E821D826F8178856115710531F0A6
:104440004B855C85872D962D0E94D217872D962D42
:104450000E949813872D962D0E94FC14B0E5EB2E38
:10446000B7E0FB2E70E060E08B010F5F1F4F809183
:10447000B0029091B102681779070CF0B801872D4E
:10448000962D0E94A317672D762DC7010E948716CF
:10449000872D962D0E94FC1426E0E20EF11CB80137
:1044A0000530110509F71093B7020093B60281E0B9
:1044B0008093B5028093B40245E050E061E00E9431
:1044C000220E2091B6023091B70200E04091B40272
:1044D0006091B5028091BE029091BF020E9434119A
:1044E000CE0107960E94FC14B2CE0E948C196AE19C
:1044F0007EE0872D962D0E946B17872D962D0E94AA
:104500009813872D962D0E94FC146FE07EE080E5C5
:1045100097E00E94431762E07EE086E597E00E9404
:10452000431782E090E09093B7028093B602109216
:10453000B5021092B40242E050E060E0FECE0E946C
:104540008C196DEF7DE0872D962D0E946B17872DBE
:10455000962D0E949813872D962D0E94FC146FEEC5
:104560007DE080E597E00E94431760EE7DE0D5CFC7
:1045700061ED7DE082E397E00E94431766EC7DE009
:1045800088E397E00E94431760917E0270917F025A
:10459000872D962D0E94FD17672D762D88E397E0D5
:1045A0000E941217872D962D0E94FC1460EC7DE06E
:1045B00088E397E00E94E8166FEA7DE08EE397E0DB
:1045C0000E94431761EA7DE084E497E00E9443176C
:1045D00060917C0270917D02872D962D0E94FD17BF
:1045E000672D762D84E497E00E941217872D962D73
:1045F0000E94FC1484E090E090937B0280937A0206
:10460000109279020E94091382E4809379078093C3
:10461000780787E380937A0768EB7CE084E797E08C
:104620000E94D40E83E490E00E94FF0F87E690E0A2
:104630000E94FF0F0CCE0E94EB306B017C0166EAFA
:104640007CE082E397E00E9443176FE97CE088E317
:1046500097E00E94431788E090E09093B302809324
:10466000B20283E090E090937B0280937A021092F2
:104670007902C701B60122E030E040E050E00E943C
:10468000EE32672B79F46AE97CE088E397E00E94D8
:10469000E81661E97CE08EE397E00E9443170E94F0
:1046A0000913D5CD6AE87CE088E397E00E94E8161C
:1046B00060E87CE08EE397E00E94431780917C02E3
:1046C00090917D02039790937D0280937C0218164F
:1046D00019062CF362E77CE084E497E00E9443171C
:1046E00084E090E090937B0280937A0288E190E0EE
:1046F0009093B3028093B202D2CF6FE87DE082E361
:1047000097E00E94431761E87DE088E397E00E940C
:1047100043176FE67DE08EE397E00E9443176BE658
:104720007DE084E497E00E94431784E090E090935A
:104730007B0280937A02109279020E9409130E94F0
:10474000F51282E090E09093B3028093B2027FCDA5
:104750000E9409138091BC029091BD020B9709F44D
:1047600076CD0E94F51273CD6AE671E082E397E0A0
:104770000E94F31761E871E088E397E00E94F31765
:1047800066E971E08EE397E00E94F3176DEA71E04D
:1047900084E497E00E94F31764EC71E08AE497E008
:1047A0000E94F31785E090E090937B0280937A0259
:1047B00081E0809379020E94091380E190E0C3CFE9
:1047C00064E671E082E397E00E94F31768ED71E020
:1047D00088E397E00E94F31767EE71E08EE397E0BD
:1047E0000E94F31783E090E090937B0280937A021B
:1047F000109279020E94091388E190E0A4CF64E648
:104800007DE0429711F06EE57DE082E397E00E9443
:1048100043176091770270917802872D962D0E9440
:104820007417672D762D82E397E00E941217872D6B
:10483000962D0E94FC146AE67DE088E397E00E94D2
:10484000431769E67DE08EE397E00E94431780916D
:10485000BC029091BD026FE47DE0429711F069E4E3
:104860007DE084E497E00E94431765E57DE08AE4FB
:1048700097E00E94431785E090E090937B0280933D
:104880007A0281E0809379020E940913E091770215
:10489000F0917802EE0FFF1FEE0FFF1FE058FD4F63
:1048A00020813181428153816091360770913707B1
:1048B000E5E0E69FC001E79F900D11246AE070E0FB
:1048C0000F960E948D148091BC029091BD02429778
:1048D000E9F4209173023091740240917502509175
:1048E00076026EE270E087E390E00E948D140E94F1
:1048F000B01465E47DE0872D962D0E946B17872DFF
:10490000962D0E945A14872D962DECCD87E3809327
:104910008307809382078EE280938407E091770279
:10492000F0917802EE0FFF1FEE0FFF1FE856FD4FCC
:1049300040815181628173818EE797E00E94FF136D
:10494000D6CF6AE37DE08431910559F06DE27DE0D8
:104950008531910531F06FE17DE0469711F060E11E
:104960007DE082E397E00E94431764E47DE088E302
:1049700097E00E94431763E47DE08EE397E00E9496
:1049800043178091B2029091B3026FEF7CE00697DB
:1049900011F067EF7CE084E497E00E94431767E042
:1049A0007DE08AE497E00E94431785E090E09093D1
:1049B0007B0280937A0281E0809379020E9409133E
:1049C0008091B2029091B3020697F9F420916F02A0
:1049D00030917002409171025091720265E270E074
:1049E00082E390E00E948D14209173023091740252
:1049F00040917502509176026EE270E087E390E09C
:104A00000E948D1463EF7CE076CF20916B02309191
:104A10006C0240916D0250916E02E0CF10927902CB
:104A200083E090E090937B0280937A021092B3022D
:104A30001092B20280906B0290906C02A0906D0276
:104A4000B0906E0280916F0290917002A0917102FD
:104A5000B0917202881A990AAA0ABB0A809173025D
:104A600090917402A0917502B0917602880E991E01
:104A7000AA1EBB1EE8E9F2E000E812E060EBE62EB9
:104A800062E0F62E2191319141915191D8016D91C1
:104A90007D918D919D918D010E94FA34860E971E15
:104AA000A81EB91EEE16FF0669F7B7FC89C08092F2
:104AB000730290927402A0927502B0927602809175
:104AC000730290917402A0917502B09176022091C8
:104AD000B8023091B90211E02F31310509F079C0E7
:104AE0004091050150910601609107017091080104
:104AF000481759076A077B070CF010E061EE7CE06D
:104B000082E397E00E94431760EE7CE088E397E041
:104B10000E9443176FEC7CE0111102C06EEC7CE048
:104B20008EE397E00E94431764ED7CE08EE397E00C
:104B30000E94E8160E9409132091730230917402BA
:104B4000409175025091760263E170E08AE090E056
:104B50000E948D148091B8029091B9024F9709F08C
:104B600041C020910501309106014091070150910B
:104B7000080167E270E08AE090E00E948D14112342
:104B800009F465CB8091730290917402A091750233
:104B9000B09176022091B8023091B9022F313105DF
:104BA00051F58093050190930601A0930701B093FE
:104BB000080165E071E086E190E00E942F1647CB86
:104BC0001092730210927402109275021092760283
:104BD00076CF4091010150910201609103017091E3
:104BE000040186CF2091010130910201409103011F
:104BF00050910401BECF8093010190930201A093D4
:104C00000301B093040161E071E08AE190E0D5CF47
:104C100085E090E090935302809352029093550266
:104C20008093540267EC7CE088E897E00E94D40E01
:104C30004091BC025091BD02052E000C660B770B13
:104C400088E897E00E94FF1302CB80E80E94320FB1
:104C500081111AC080E10E94320F811115C080E2DB
:104C60000E94320F811110C080E40E94320F811126
:104C70000BC088E00E94320F811106C084E00E94C0
:104C8000320F882309F466C0A090B602B090B70234
:104C9000E090B402ED86E090BE02F090BF0201E029
:104CA00095014D856091B502C7010E943411B5018F
:104CB0000B2C000C880B990B0E94BB3120E030E0DC
:104CC00040E05FE30E941A321B012C0120E030E03B
:104CD000A9010E94F53420E030E040E05FE387FD69
:104CE0003DC0C201B1010E9489330E9467348B012B
:104CF00088248394912CE616F7061CF042E0842E5B
:104D0000912C80E10E94320F8823A9F10FEFE01A65
:104D1000F00AEA14FB043CF5F092BF02E092BE02F6
:104D2000E090BE02F090BF022091B6023091B7022F
:104D300000E04091B4026091B502C7010E943411B5
:104D40008091BC029091BD020497029718F4C701AC
:104D50000E94341980E00E940508EEC8C201B1012A
:104D60000E948833C2CF11E0A11AB108B092BF02ED
:104D7000A092BE02D5CF80E80E94320F882371F046
:104D800021E0E21AF108F092BF02E092BE02F7FEC3
:104D9000C7CF1092BF021092BE02C2CF80E40E9421
:104DA000320F8823E1F0CD84CC20A9F08A948928A1
:104DB00091F4E00EF11EF092BF02E092BE028091EB
:104DC000BE029091BF028A159B050CF4A9CF41E069
:104DD000A41AB108CBCF3FEFE31AF30AECCF80E27D
:104DE0000E94320F8823C1F0CD84CC2089F022E0CC
:104DF0008216910469F4E01AF10AF092BF02E0927F
:104E0000BE028091BE029091BF0297FF89CFC1CFB1
:104E100031E0E31AF108F1CF88E00E94320F8823D5
:104E200009F42CC51092C20248E0C416D10408F05F
:104E300077CFF601E25EF84D0C940A3526279026CE
:104E40005A278627852A4B2BAD2B0B2C81E0E816A1
:104E5000F10461F092E0E916F10459F08EE190E07E
:104E6000EF2809F05DCF0E94DF155ACF8CE390E068
:104E7000FACF65E67CE082E397E00E94431764E6A0
:104E80007CE088E397E00E94431765E57CE08EE3D1
:104E900097E00E9443171092790283E090E090938C
:104EA0007B0280937A0281E090E09093BD02809330
:104EB000BC0236CF82E090E09093B3028093B202BE
:104EC000A2E0EA16F104C9F04CF4E114F10491F007
:104ED00085E090E0EA94EF2841F322CFF4E0EF166A
:104EE000F10489F06CF087E090E015E0E116F10440
:104EF000E1F216CF84E090E0D8CF8AE090E0D5CF01
:104F000083E090E0D2CF86E090E0CFCF8091B002F6
:104F10009091B102E816F9061CF02FEFE21AF20A9E
:104F2000F092B102E092B00281E00E9404150E946A
:104F3000EB3024E130E040E050E00E94EE329B0193
:104F400042E050E05093B3024093B20210927902D3
:104F5000FB013197E131F10508F0D2C2EE54F84D72
:104F60000C940A35C327EA2709283C283C286728DF
:104F700067289428DB28DB28DB283B293B298F295D
:104F8000B029DF294D2A6CEC7BE082E397E00E9498
:104F900043176EEB7BE088E397E00E94431765EBD5
:104FA0007BE08EE397E00E94431783E090E09093CC
:104FB0007B0280937A0282E090E0A0E0B0E08093F0
:104FC000940290939502A0939602B09397028BE07F
:104FD00090E06BCF64EA7BE082E397E00E944317A6
:104FE00064E97BE088E397E00E94431782E090E069
:104FF00090937B0280937A028AE790E0A0E0B0E091
:1050000080938C0290938D02A0938E02B0938F02B6
:10501000DECF63E87BE082E397E00E94431765E719
:105020007BE088E397E00E94431764E67BE08EE331
:1050300097E00E9443176BE57BE084E497E00E94D1
:10504000431784E090E090937B0280937A020E9461
:10505000EB302EE734E040E050E00E94EE326E5A32
:105060007C4F8F4F9F4F6093840270938502809393
:10507000860290938702ABCF6FE47BE082E397E0F8
:105080000E94431760E47BE088E397E00E944317A7
:1050900062E37BE08EE397E00E94431768E27BE0E7
:1050A00084E497E00E94431784E090E090937B02B1
:1050B00080937A020E94EB3029EA31E640E050E02A
:1050C0000E94EE32605B794B8F4F9F4FCCCF68E1EF
:1050D0007BE082E397E00E94431766E07BE088E391
:1050E00097E00E94431763EF7AE08EE397E00E9417
:1050F000431783E090E090937B0280937A020E94B2
:10510000EB3021E63AEE40E050E00E94EE3260588B
:10511000774C8E4F9F4F60938002709381028093F3
:1051200082029093830253CF63EE7AE082E397E0AA
:105130000E94431764ED7AE088E397E00E944317EA
:1051400082E090E090937B0280937A0260917302F8
:105150007091740280917502909176020E94BB3129
:1051600020E030E040E450E40E94F5336B017C0124
:1051700020E030E0A9010E94F53420E030E040E07A
:105180005FE387FD13C0C701B6010E9489330E9407
:105190006734660F771F881F991F6093730270939F
:1051A0007402809375029093760211CFC701B60105
:1051B0000E948833ECCFE8E9F2E090E080E0419192
:1051C000519161917191840F951FA2E0E03BFA0724
:1051D000B1F7C2970CF468C382E090E02930310542
:1051E00039F084E090E02A30310511F085E090E05C
:1051F00090937F0280937E0264EC7AE082E397E0F2
:105200000E9443176FEB7AE088E397E00E94431710
:1052100060917E0270917F0261507109872D962DF9
:105220000E94FD17672D762D88E397E00E941217E4
:10523000872D962D0E94FC1467EB7AE088E397E0B7
:105240000E94E8166AEA7AE08EE397E00E9443172C
:105250006FE97AE084E497E00E94431784E090E0ED
:1052600090937B0280937A0288E090E09093B3025F
:105270008093B202ACCE8091730290917402A0919F
:105280007502B0917602843F9140A105B1050CF4FE
:105290000BC30E947C1205970CF406C30E94EB30EE
:1052A00023E030E040E050E00E94EE326B0160E924
:1052B0007AE082E397E00E944317F2E0CF16D10430
:1052C000C8F467E77AE0CD2811F068E67AE088E371
:1052D00097E00E94431763E87AE08EE397E00E942C
:1052E000431783E090E090937B0280937A028CE0F6
:1052F00090E0DBCD69E57AE088E397E00E94431710
:1053000069E47AE08EE397E00E94431760E47AE074
:1053100084E497E00E94431784E090E0E4CF6EE2DB
:105320007AE082E397E00E9443176DE17AE088E338
:1053300097E00E9443176BE07AE08EE397E00E94CB
:10534000431768EF79E084E497E00E94431784E014
:1053500090E090937B0280937A028EE090E0A5CD5E
:105360008091730290917402A0917502B0917602BF
:105370008C329140A105B1050CF496C265EE79E03E
:1053800082E397E00E94431765ED79E088E397E0B8
:105390000E94431764EC79E08EE397E00E94431784
:1053A00069EB79E084E497E00E94431784E090E0A1
:1053B00090937B0280937A028DE090E076CD0E94FC
:1053C0007C1208970CF470C20E94EB3027E030E0AA
:1053D00040E050E00E94EE328B010F5F1F4F0E94B1
:1053E000EB3026E030E040E050E00E94EE326B010E
:1053F000FB01EE0FFF1FEE0FFF1FE856FD4FA80148
:10540000012E000C660B770B80819181A281B38104
:10541000840F951FA61FB71F80839183A283B38338
:105420006EEA79E082E397E00E944317B801872D86
:10543000962D0E94FD17672D762D82E397E00E943E
:105440001217872D962D0E94FC1463EA79E088E3F9
:1054500097E00E944317B601872D962D0E9474177E
:10546000672D762D88E397E00E941217872D962DE1
:105470000E94FC1465EF71E08EE397E00E94F31741
:1054800067E072E084E497E00E94F31784E090E024
:1054900090937B0280937A029ACD65E172E082E379
:1054A00097E00E94F31764E272E088E397E00E94BD
:1054B000F31766E372E08EE397E00E94F31765E46A
:1054C00072E084E497E00E94F31784E090E0909308
:1054D0007B0280937A020E94EB3027E232E040E0C8
:1054E00050E00E94EE3266507F4F8F4F9F4F609387
:1054F00088027093890280938A0290938B0267CD11
:105500005093BD024093BC020BCC0E947C128C01D4
:1055100094E0C92ED12CD092B302C092B202F09284
:105520007802E092770210161106DCF16FE47CE05D
:1055300082E397E00E9443176EE47CE088E397E003
:105540000E9443176EE37CE08EE397E00E944317CE
:1055500068E37CE084E497E00E944317609177025F
:1055600070917802872D962D0E947417672D762DE5
:1055700084E497E00E941217872D962D0E94FC1458
:1055800066E37CE084E497E00E94E816D0927B0218
:10559000C0927A02109279028091BC029091BD0271
:1055A00065CEF701EE0FFF1FEE0FFF1FE058FD4F16
:1055B00080809180A280B3806091730270917402A8
:1055C0008091750290917602681579058A059B0590
:1055D0003CF560E37CE082E397E00E9443176FE2D2
:1055E0007CE088E397E00E9443176EE17CE08EE365
:1055F00097E00E9443176091770270917802872D9F
:10560000962D0E947417672D762D84E497E00E94F2
:105610008716872D962D0E94FC146CE17CE0B2CF9A
:1056200022E130E03093BD022093BC02109263026D
:105630001092640210926502109266020E94BB31C1
:105640006B017C01C501B4010E94BB319B01AC011F
:10565000C701B6010E94F5330E949D340E94673451
:10566000609358027093590280935A0290935B02A0
:10567000012E000C220B330B0617170728073907DA
:105680000CF04ECB009358021093590220935A020B
:1056900030935B0245CB85E090E09093B30280931A
:1056A000B202F0927802E0927702F701EE0FFF1F4C
:1056B000EE0FFF1FE856FD4F80819181A281B381DB
:1056C000181619061A061B06BCF423E130E03093C5
:1056D000BD022093BC0210926302109264021092E9
:1056E0006502109266028093580290935902A0932B
:1056F0005A02B0935B0214CB66E17CE082E397E050
:105700000E94431765E17CE088E397E00E9443171D
:1057100062E07CE08EE397E00E944317609177029D
:1057200070917802872D962D0E947417672D762D23
:1057300084E497E00E948716872D962D0E94FC1422
:1057400060E07CE084E497E00E94E81684E090E06A
:1057500090937B0280937A021DCF86E090E0909335
:10576000B3028093B202109263021092640210920C
:10577000650210926602E114F10419F1EA94EF282F
:1057800009F0CECA809162028823D1F164EF7BE0F8
:1057900082E397E00E94431765EE7BE088E397E0A1
:1057A0000E9443176EED7BE08EE397E00E94431763
:1057B00083E090E090937B0280937A0210927902CA
:1057C00006CC84E190E09093BD028093BC024091AE
:1057D000730250917402609175027091760280910B
:1057E0006F0290917002A0917102B09172024817FD
:1057F00059076A077B070CF076CFDB01CA0173CF2C
:1058000085E190E09093BD028093BC0288E893E12B
:10581000A0E0B0E068CF87E090E09093B30280937F
:10582000B20210926302109264021092650210920A
:105830006602E114F10499F0EA94EF2809F070CAC5
:1058400087E190E09093BD028093BC0280916B024F
:1058500090916C02A0916D02B0916E0244CF86E1EE
:1058600090E09093BD028093BC028091730290916E
:105870007402A0917502B091760235CF84E00E9447
:10588000320F882309F44CCAA3E0CA1AD108B5E044
:10589000CB16D10408F044CA1092C2020E949212A0
:1058A0009093C1028093C00282E090E0FECA81E042
:1058B0000E94D4124FCA80E00E94D41281114ACAB9
:1058C00088E00E94320F882309F444CA1092C20271
:1058D0008091BC029091BD028D30910509F44EC0BB
:1058E00060F50C9709F036CA8091690290916A02BE
:1058F000019690936A02809369028091730290915D
:105900007402A0917502B091760280599140A1096C
:10591000B1098093730290937402A0937502B093BF
:1059200076028091670290916802059790936802D1
:105930008093670282E090E041C08E309105E1F1F2
:10594000419709F007CA8091730290917402A09167
:105950007502B0917602885E9340A109B1098093E7
:10596000730290937402A0937502B093760282E35F
:1059700090E090937D0280937C02DCCF809167025F
:10598000909168020A9690936802809367028091D2
:10599000730290917402A0917502B0917602885CB6
:1059A0009109A109B1098093730290937402A093A5
:1059B0007502B0937602BECF8FE090E09093BD0267
:1059C0008093BC02C7C984E00E94320F882309F487
:1059D00040C01092C2020E94EB3022E030E040E072
:1059E00050E00E94EE32672B682B692BD9F462E9F4
:1059F00079E082E397E00E94431767E879E088E363
:105A000097E00E94431782E090E090937B0280939E
:105A10007A02109279029093B3028093B2028BE0E3
:105A200090E0CCCF67E779E082E397E00E944317EC
:105A300061E779E088E397E00E94431782E090E015
:105A400090937B0280937A021092790289E090E031
:105A5000E2CF88E00E94320F882309F47BC91092BC
:105A6000C2028091690290916A02892BE9F462E690
:105A700079E082E397E00E94431764E579E088E3E8
:105A800097E00E94431767E479E08EE397E00E9475
:105A9000431783E090E090937B0280937A02109208
:105AA000790288E090E0B7CF0E94EB3022E030E04E
:105AB00040E050E00E94EE32672B682B692B49F4DE
:105AC00066E479E082E397E00E94431766E379E0B9
:105AD000B1CF80917E0290917F02019790937F02D7
:105AE00080937E02181619064CF465E379E082E390
:105AF00097E00E94431764E279E09CCF0E94EB306C
:105B000023EE34E040E050E00E94EE328B0102517F
:105B10001D4F62E179E082E397E00E94431761E064
:105B200079E088E397E00E944317B801872D962D0E
:105B30000E94FD17672D762D88E397E00E941217CB
:105B4000872D962D0E94FC146EEE78E08EE397E090
:105B50000E9443176BED78E084E497E00E944317BE
:105B600084E090E090937B0280937A0281E08093BE
:105B70007902012E000C220B330B8091730290915D
:105B80007402A0917502B0917602800F911FA21F3E
:105B9000B31F8093730290937402A0937502B09325
:105BA0007602803B9440A105B1051CF081E190E0B4
:105BB00032CF82E090E02FCF80E00E94D41281119A
:105BC000C9C888E00E94320F882309F43FC1809140
:105BD000BC029091BD028431910509F4BDC098F4D6
:105BE0008231910509F47FC04397F1F11092C2020E
:105BF0000E9492129093C1028093C0028091B202DF
:105C00009091B302DBCE8631910509F402C108F40C
:105C1000CCC0479759F7409163025091640260915C
:105C200065027091660280916B0290916C02A09166
:105C30006D02B0916E02841B950BA60BB70B80937F
:105C40006B0290936C02A0936D02B0936E028091F0
:105C5000730290917402A0917502B0917602840F44
:105C6000951FA61FB71F36C08091770290917802CA
:105C70002091630230916402409165025091660266
:105C8000880F991F880F991FFC01E856FD4FC080AF
:105C9000D180E280F380C21AD30AE40AF50AC082F6
:105CA000D182E282F38280589D4FDC016D917D911B
:105CB0008D919C910E94FA340091730210917402AC
:105CC0002091750230917602DC01CB01800F911F8B
:105CD000A21FB31F8093730290937402A093750266
:105CE000B093760283CF80917702909178022091D1
:105CF0006302309164024091650250916602880F00
:105D0000991F880F991FFC01E856FD4FC080D18074
:105D1000E280F380C20ED31EE41EF51EC082D18243
:105D2000E282F38280589D4FFC0160817181828103
:105D300093810E94FA3400917302109174022091B1
:105D400075023091760268017901C61AD70AE80A0D
:105D5000F90AD701C601BECF409163025091640297
:105D6000609165027091660280916F02909170025D
:105D7000A0917102B0917202841B950BA60BB70B18
:105D800080936F0290937002A0937102B09372029D
:105D90008091730290917402A0917502B091760285
:105DA000841B950BA60BB70B95CF409163025091C6
:105DB0006402609165027091660280916F02909119
:105DC0007002A0917102B0917202840F951FA61FFC
:105DD000B71F80936F0290937002A0937102B093EB
:105DE00072028091730290917402A0917502B09139
:105DF0007602840F951FA61FB71F8093730290939E
:105E00007402A0937502B093760281E080936202DF
:105E1000EDCE4091630250916402609165027091F1
:105E2000660280916B0290916C02A0916D02B0911C
:105E30006E02840F951FA61FB71F80936B0290936D
:105E40006C02A0936D02B0936E02A2CF8FB7F8944C
:105E50008090C4029090C502A090C602B090C70284
:105E60008FBF8091BC029091BD024297C12CD12C72
:105E70007601C394029728F07AE0C72ED12CE12C4A
:105E8000F12C80915E0290915F02A0916002B0912E
:105E9000610295018401081B190B2A0B3B0B8091B1
:105EA0005C0290915D0244EF51E060E070E082306E
:105EB000910554F044E650E060E070E085319105D2
:105EC0001CF040E050E0BA01401751076207730729
:105ED00010F00C94AA26843691050CF45CC05AE0AC
:105EE000252E312C412C512C8D379105BCF044E6E8
:105EF000242E312C412C512C863991057CF068EEF2
:105F0000262E63E0362E412C512C8F3A910534F029
:105F100030E1232E37E2332E412C512C883E03E012
:105F200090072CF4019690935D0280935C020E948E
:105F30002A0F87FF41C080925E0290925F02A0927A
:105F40006002B092610240915802509159026091F2
:105F50005A0270915B028091630290916402A09159
:105F60006502B09166028A019B010C191D092E0978
:105F70003F09081719072A073B0794F08C0D9D1D50
:105F8000AE1DBF1D8093630290936402A0936502CF
:105F9000B09366020DC0212C312C21012394C2CF75
:105FA00040936302509364026093650270936602AB
:105FB0000E94B0140C94AA260E942A0F86FF39C0B2
:105FC00080925E0290925F02A0926002B0926102A3
:105FD000AAE0B0E0A70196010E940D339B01AC013D
:105FE000C201B1010E94FA3400916302109164026F
:105FF0002091650230916602DC01CB01800F911F78
:10600000A21FB31F009158021091590220915A0209
:1060100030915B02081719072A073B070CF0B2CF33
:10602000009363021093640220936502309366022A
:10603000BFCF0E942A0F84FF23C080925E029092FD
:106040005F02A0926002B09261028091630290911F
:106050006402A0916502B09166028C159D05AE05A3
:10606000BF052CF08C199D09AE09BF098BCF10928A
:10607000630210926402109265021092660298CF39
:106080000E942A0F85FF2AC080925E0290925F02D2
:10609000A0926002B0926102AAE0B0E0A70196016E
:1060A0000E940D339B01AC01C201B1010E94FA3480
:1060B00000916302109164022091650230916602A2
:1060C000061717072807390794F268017901C61ADD
:1060D000D70AE80AF90AD701C60154CF10925E0226
:1060E00010925F02109260021092610210925D02A3
:1060F00010925C020C94AA26CF93DF938AE497E077
:106100000E94FC1484E497E00E94FC148EE397E064
:106110000E94FC1488E397E00E94FC1482E397E05D
:106120000E94FC14C4E7D7E02697CE010E94FC141D
:1061300087E0C035D807C1F7DF91CF9108958F92DE
:106140009F92AF92BF92CF92DF92EF92FF92CF9346
:10615000DF93EC01688179818A819B8161157105EA
:106160008105910521F464E279ED8BE597E02DE15D
:1061700033EF41E050E00E94EE3249015A019B01A9
:10618000AC01A7EAB1E40E940D336B017C01ACEED7
:10619000B4EFA50194010E941B33C60ED71EE81E62
:1061A000F91EF7FE06C081E0C81AD108E10880E8B0
:1061B000F80AC882D982EA82FB82C701B6019F77BA
:1061C000DF91CF91FF90EF90DF90CF90BF90AF9095
:1061D0009F908F9008958F929F92AF92BF92CF928F
:1061E000DF92EF92FF9260911501709116018091FC
:1061F000170190911801611571058105910521F430
:1062000064E279ED8BE597E02DE133EF41E050E07A
:106210000E94EE3249015A019B01AC01A7EAB1E4A8
:106220000E940D336B017C01ACEEB4EFA50194012B
:106230000E941B33C60ED71EE81EF91EF7FE06C0CD
:1062400081E0C81AD108E10880E8F80AC092150177
:10625000D0921601E0921701F0921801C701B60121
:106260009F77FF90EF90DF90CF90BF90AF909F907F
:106270008F90089560931501709316018093170114
:10628000909318010895FB01DC0105900D92002008
:10629000E1F70895FC0105900020E9F780959095BD
:1062A0008E0F9F1F0895BB274A3031F4992322F4A3
:1062B000BDE2909581959F4F0C949031BB272A3079
:1062C00051F4992342F4BDE29095809570956195C3
:1062D0007F4F8F4F9F4F0C946E31BB27FA01A62F33
:1062E0006217710581059105330B30FB66F0AA2713
:1062F000660F771F881F991FAA1FA21710F0A21BF5
:1063000063953850A9F7A05DAA3308F0A95DA19361
:1063100036F7B111B1931082CA010C94A931BB2791
:10632000FB015527AA27880F991FAA1FA41710F051
:10633000A41B83955051B9F7A05DAA3308F0A95D5D
:10634000A193009779F7B111B1931192CB010C94FD
:10635000A931DC01FC01672F71917723E1F73297B6
:1063600004C07C916D9370836291AE17BF07C8F330
:106370000895E89409C097FB3EF490958095709538
:1063800061957F4F8F4F9F4F9923A9F0F92F96E981
:10639000BB279395F695879577956795B795F111F6
:1063A000F8CFFAF4BB0F11F460FF1BC06F5F7F4F93
:1063B0008F4F9F4F16C0882311F096E911C07723A5
:1063C00021F09EE8872F762F05C0662371F096E8AE
:1063D000862F70E060E02AF09A95660F771F881F7D
:1063E000DAF7880F9695879597F90895990F000821
:1063F000550FAA0BE0E8FEEF16161706E807F90797
:10640000C0F012161306E407F50798F0621B730B31
:10641000840B950B39F40A2661F0232B242B252BB2
:1064200021F408950A2609F4A140A6958FEF811D55
:10643000811D08950E942D320C949E320E9490324C
:1064400038F00E94973220F0952311F00C94873297
:106450000C948D3211240C94D2320E94AF3270F31E
:10646000959FC1F3950F50E0551F629FF001729FF9
:10647000BB27F00DB11D639FAA27F00DB11DAA1F08
:10648000649F6627B00DA11D661F829F2227B00D55
:10649000A11D621F739FB00DA11D621F839FA00DE0
:1064A000611D221F749F3327A00D611D231F849F30
:1064B000600D211D822F762F6A2F11249F57504087
:1064C0009AF0F1F088234AF0EE0FFF1FBB1F661F02
:1064D000771F881F91505040A9F79E3F510580F0CB
:1064E0000C9487320C94D2325F3FE4F3983ED4F39D
:1064F000869577956795B795F795E7959F5FC1F76F
:10650000FE2B880F911D9695879597F9089597F919
:106510009F6780E870E060E008959FEF80EC089549
:1065200000240A9416161706180609060895002472
:106530000A9412161306140605060895092E0394EC
:10654000000C11F4882352F0BB0F40F4BF2B11F460
:1065500060FF04C06F5F7F4F8F4F9F4F089557FDBF
:106560009058440F551F59F05F3F71F04795880FC1
:1065700097FB991F61F09F3F79F087950895121658
:1065800013061406551FF2CF4695F1DF08C0161604
:1065900017061806991FF1CF8695710561050894B5
:1065A0000895E894BB2766277727CB0197F90895CC
:1065B000F999FECF92BD81BDF89A992780B50895CB
:1065C000262FF999FECF1FBA92BD81BD20BD0FB60F
:1065D000F894FA9AF99A0FBE01960895052E97FB42
:1065E0001EF400940E94053357FD07D00E945733D4
:1065F00007FC03D04EF40C9405335095409530952C
:1066000021953F4F4F4F5F4F08959095809570951E
:1066100061957F4F8F4F9F4F08950E947933A59FBB
:10662000900DB49F900DA49F800D911D112408958D
:10663000B7FF0C940D330E940D33821B930B08950A
:106640002F923F924F925F926F927F928F929F9282
:10665000AF92BF92CF92DF92EF92FF920F931F9370
:10666000CF93DF93CDB7DEB7CA1BDB0B0FB6F89421
:10667000DEBF0FBECDBF09942A88398848885F8461
:106680006E847D848C849B84AA84B984C884DF80D2
:10669000EE80FD800C811B81AA81B981CE0FD11DB6
:1066A0000FB6F894DEBF0FBECDBFED010895A1E295
:1066B0001A2EAA1BBB1BFD010DC0AA1FBB1FEE1F7C
:1066C000FF1FA217B307E407F50720F0A21BB30BC7
:1066D000E40BF50B661F771F881F991F1A9469F743
:1066E00060957095809590959B01AC01BD01CF019F
:1066F0000895A29FB001B39FC001A39F700D811D9B
:106700001124911DB29F700D811D1124911D0895BA
:106710005058BB27AA270E94A0330C949E320E9497
:10672000903238F00E94973220F039F49F3F19F4EC
:1067300026F40C948D320EF4E095E7FB0C9487322E
:10674000E92F0E94AF3258F3BA1762077307840724
:10675000950720F079F4A6F50C94D1320EF4E0956B
:106760000B2EBA2FA02D0B01B90190010C01CA010B
:10677000A0011124FF27591B99F0593F50F4503EB6
:1067800068F11A16F040A22F232F342F4427585FA8
:10679000F3CF469537952795A795F0405395C9F7C0
:1067A0007EF41F16BA0B620B730B840BBAF0915078
:1067B000A1F0FF0FBB1F661F771F881FC2F70EC017
:1067C000BA0F621F731F841F48F4879577956795EA
:1067D000B795F7959E3F08F0B0CF9395880F08F0D6
:1067E0009927EE0F9795879508950E9409340C9488
:1067F0009E320E94973258F00E94903240F029F465
:106800005F3F29F00C94873251110C94D2320C94D2
:106810008D320E94AF3268F39923B1F3552391F37F
:10682000951B550BBB27AA2762177307840738F0FF
:106830009F5F5F4F220F331F441FAA1FA9F335D05C
:106840000E2E3AF0E0E832D091505040E695001C10
:10685000CAF72BD0FE2F29D0660F771F881FBB1FCA
:10686000261737074807AB07B0E809F0BB0B802DA8
:10687000BF01FF2793585F4F3AF09E3F510578F0D4
:106880000C9487320C94D2325F3FE4F3983ED4F3F9
:10689000869577956795B795F7959F5FC9F7880FA8
:1068A000911D9695879597F90895E1E0660F771FFA
:1068B000881FBB1F621773078407BA0720F0621B8B
:1068C000730B840BBA0BEE1F88F7E09508950E94B6
:1068D0006E346894B1110C94D23208950E94B7328C
:1068E00088F09F5798F0B92F9927B751B0F0E1F091
:1068F000660F771F881F991F1AF0BA95C9F714C041
:10690000B13091F00E94D132B1E008950C94D132AF
:10691000672F782F8827B85F39F0B93FCCF3869579
:1069200077956795B395D9F73EF4909580957095D6
:1069300061957F4F8F4F9F4F08950E94DD3490F0F7
:106940009F3748F4911116F00C94D23260E070E059
:1069500080E89FEB089526F41B16611D711D811DB3
:106960000C94B4340C94CF34882371F4772321F041
:106970009850872B762F07C0662311F499270DC0F6
:106980009051862B70E060E02AF09A95660F771F91
:10699000881FDAF7880F9695879597F908959F3F96
:1069A00031F0915020F4879577956795B795880FCA
:1069B000911D9695879597F908950E94B732A0F09A
:1069C000BEE7B91788F4BB279F3860F41616B11DCF
:1069D000672F782F8827985FF7CF869577956795EB
:1069E000B11D93959639C8F308950E94F63108F4C5
:1069F0008FEF0895DB018F939F930E940D33BF911A
:106A0000AF91A29F800D911DA39F900DB29F900DFD
:106A100011240895EE0FFF1F0590F491E02D0994C5
:106A20000F931F93CF93DF938230910510F482E090
:106A300090E0E0918E07F0918F0730E020E0B0E029
:106A4000A0E0309799F42115310509F44AC0281BBC
:106A5000390B24303105D8F58A819B816115710588
:106A600089F1FB0193838283FE0111C04081518132
:106A70000281138148175907E0F04817590799F424
:106A8000109761F012960C93129713961C933296FE
:106A9000CF01DF91CF911F910F91089500938E0741
:106AA00010938F07F4CF2115310551F0421753078A
:106AB00038F0A901DB019A01BD01DF01F801C1CF66
:106AC000EF01F9CF90938F0780938E07CDCFFE0112
:106AD000E20FF31F81939193225031093983288368
:106AE000D7CF20918C0730918D07232B41F4209133
:106AF0001B0130911C0130938D0720938C0720914E
:106B0000190130911A012115310541F42DB73EB715
:106B100040911D0150911E01241B350BE0918C0703
:106B2000F0918D07E217F307A0F42E1B3F0B2817F7
:106B3000390778F0AC014E5F5F4F2417350748F0F6
:106B40004E0F5F1F50938D0740938C078193919355
:106B50009FCFF0E0E0E09CCFCF93DF930097E9F088
:106B6000FC01329713821282A0918E07B0918F0799
:106B7000ED0130E020E01097A1F420813181820FF7
:106B8000931F20918C0730918D072817390709F042
:106B900061C0F0938D07E0938C07DF91CF9108954A
:106BA000EA01CE17DF07E8F54A815B819E014115B6
:106BB0005105B1F7E901FB83EA8349915991C40F6B
:106BC000D51FEC17FD0761F4808191810296840F37
:106BD000951FE90199838883828193819B838A83AE
:106BE000F0E0E0E012968D919C9113970097B9F533
:106BF0002D913C911197CD010296820F931F209108
:106C00008C0730918D072817390739F6309751F5E1
:106C100010928F0710928E07B0938D07A0938C0768
:106C2000BCCFD383C28340815181840F951FC81785
:106C3000D90761F44E5F5F4F88819981480F591FD2
:106C4000518340838A819B819383828321153105FF
:106C500009F0B0CFF0938F07E0938E079ECFFD0130
:106C6000DC01C0CF13821282D7CFB0E0A0E0EBE30B
:106C7000F6E30C9422338C01009751F4CB010E946F
:106C800010358C01C801CDB7DEB7E0E10C943E337E
:106C9000FC01E60FF71F9C0122503109E217F307B0
:106CA00008F49DC0D901CD91DC911197C617D70783
:106CB00098F0C530D10530F3CE01049786179707B9
:106CC00008F3C61BD70B2297C193D1936D937C9386
:106CD000CF010E94AC35D6CF5B01AC1ABD0A4C0186
:106CE0008C0E9D1EA0918E07B0918F07512C412CC8
:106CF000F12CE12C109731F580918C0790918D0744
:106D00008815990509F05CC04616570608F058C06A
:106D10008091190190911A01009741F48DB79EB7A7
:106D200040911D0150911E01841B950BE817F90736
:106D300008F055C0F0938D07E0938C07F90171833B
:106D40006083A0CF8D919C91119712966C901297B1
:106D500013967C901397A815B90559F56C0142E07C
:106D6000C40ED11CCA14DB0420F1AC014A195B0922
:106D7000DA011296159780F0628273825183408304
:106D8000D9016D937C93E114F10471F0D70113964E
:106D9000FC93EE93129776CF22968C0F9D1FF901EC
:106DA00091838083F301EFCFF0938F07E0938E07F9
:106DB00069CF4816590608F42C017D01D3019ACFFA
:106DC000CB010E9410357C01009749F0AE01B8015B
:106DD0000E94F236C8010E94AC35870153CF10E003
:106DE00000E050CFFB01DC0102C001900D92415048
:106DF0005040D8F70895FB01DC018D910190801976
:106E00000110D9F3990B0895FB01DC0101900D925B
:106E10000020E1F7089517E0CAEDD7E004C0FE01B5
:106E20000E940A352196CB3DD107C9F7F894FFCFD0
:106E300010400D0300A0860100FFFFFFFF00E100EE
:106E4000000000000001000000000090078000002A
:106E5000C1808100000000000000230C8E0D440C56
:106E6000390C8A0C480C660C000000002E12F80E3B
:106E7000A313130E00000000E011F80EA313130E6D
:106E800000000000A810F80EA313130E596F752010
:106E90006F776E2000736C6E6700596F75206861A4
:106EA0006C6C7563696E617465206F6E20746865C3
:106EB0000077696C646573742074726970206F6602
:106EC00020796F7572006C6966652C207374756D1E
:106ED000626C65206F6E746F2074686500737562F4
:106EE00077617920747261636B732C20616E64200A
:106EF00067657400637265616D6564206279206105
:106F000020747261696E2E002020204A75737420EF
:106F1000736179206E6F0020202020746F206472CE
:106F20007567732E006F6E20612064656164206454
:106F300075646520696E0074686520737562776199
:106F40007921212100546865206D61726B65742080
:106F5000686173006265656E20666C6F6F6465645E
:106F6000207769746800636865617020686F6D657B
:0E6F70006D6164650061636964212121210067
:00000001FF
